:020000040000FA
:10000000A0EF7FF0FFFFFFFFFACF7FFF9AEF39F0FD
:10001000A6A21200FDD7FFFFD8CF64FF96EF39F0FC
:100020000AEE18F01FEE64F097EC57F000EE11F0B6
:1000300010EE13F097EC57F000EE75F011EE00F0B3
:1000400097EC57F03FEF3AF00001CF6BD06BD16BDC
:10005000D26B230ED36F0A0ED46FF0EC4DF000017B
:10006000BB6FBB05D8B402D0BB511200E5CBE8FF93
:10007000040AD8B405D0E5CBE8FF060AD8A40AD014
:1000800021CCE8FF550AD8A405D022CCE8FFAA0A63
:10009000D8B406D00001836B846B856B866B44D02B
:1000A000E9CB00F0000100C083F0846B856B866BA8
:1000B000080EEACB00F0016A026A036A6BEC57F0A3
:1000C00000EE83F00050EE260150EE220250EE22A8
:1000D0000350ED22ED52ED52100EF5CB00F0016A07
:1000E000026A036A6BEC57F000EE83F00050EE26D4
:1000F0000150EE220250EE220350ED22ED52ED525D
:10010000180EF6CB00F0016A026A036A6BEC57F036
:1001100000EE83F00050EE260150EE220250EE2257
:100120000350ED22ED52ED5283C0CFF084C0D0F0E9
:1001300085C0D1F086C0D2F00001230ED36F0A0E25
:10014000D46FF0EC4DF0006E00C002F0036A035073
:100150000210D8B41E0C23CAE8FFE90AD8B405D0AF
:1001600023CAE8FFEB0AD8A41F0C0AEE2EF0EF50CA
:10017000D8A4200C2FCAE8FF020AD8A4200C38CA41
:10018000E8FFF80AD8A4210C35CA7AF034CA79F00D
:1001900079C000F07AC001F0050ED8900036013623
:1001A000E82EFBD70006010E0122090E026ED89040
:1001B00001320032022EFBD700500001BC6F01500B
:1001C000BD6FBE6BBF6B32CA01F0006A000E01BE8C
:1001D000FF0E026E036E31CAE8FF0024046E000EAB
:1001E0000120056E000E0220066E000E0320076E31
:1001F00000EE83F00450EE260550EE220650EE226B
:100200000750ED22ED52ED523ACA01F0006A39CAA8
:10021000E8FF0024046E000E0120056E066A05BE8C
:1002200006060650076E04C0C0F005C0C1F006C047
:10023000C2F007C0C3F033CA22FAC0C004F0C1C084
:1002400005F0C2C006F0C3C007F022CA00F0016A80
:10025000026A036A84EC56F083C0E8FF0024E8CF0A
:100260007FF084C0E8FF0120E8CF80F085C0E8FF80
:100270000220E8CF81F086C0E8FF0320E8CF82F0BB
:1002800030CA21FABC0EE96E000EEA6E0001EE5093
:100290007F25E8CF7BF0EE508021E8CF7CF0EE5058
:1002A0008121E8CF7DF0ED508221E8CF7EF0ED5244
:1002B000ED52010CBE000001C36BC46BC56BC66B75
:1002C000BEC0D9FFBFC0DAFFC051D8A409D000EE2C
:1002D0000CF0D950E926DA50EA22EE6AED6AC9D16B
:1002E0000001C005D8B4BCD10001C051020AD8A495
:1002F000C0D1ACD17FC004F080C005F081C006F051
:1003000082C007F000EE0CF0D950E926DA50EA225C
:10031000EECF00F0EDCF01F0040E026ED890013266
:100320000032022EFBD7026A036A005004260150F5
:100330000522025006220350072200EE0CF0D9508D
:10034000E926DA50EA22EECF00F0EDCF01F00F0EF1
:100350000016000E0116050ED89000360136E82E64
:10036000FBD700C0C1F001C0C2F0D9CFBEF0DACFD8
:10037000BFF000010750C61908E10650C51905E194
:100380000550C41902E10450C319D8B41ED004C0EA
:10039000C3F005C0C4F006C0C5F007C0C6F0C3C0B6
:1003A000CFF0C4C0D0F0C5C0D1F0C6C0D2F0230E8B
:1003B000D36F0A0ED46FF0EC4DF0006E00C002F067
:1003C000036A03500210D8B4000CBEC0D9FFBFC0EE
:1003D000DAFF00010AEE23F0C151E926C251EA22F8
:1003E000EF50D8B42ED10AEE23F0C151E926C25104
:1003F000EA22EF50E50AD8B424D100010AEE23F036
:10040000C151E926C251EA22EF502E0AD8B419D1BF
:1004100000010AEE2EF0C151E926C251EA22EF5046
:100420001A0BD8A40ED1F36AF3500001C125006E57
:10043000000EC221016E230E0024E16E0A0E01207F
:10044000E26EF350D924E96E000EDA20EA6EE7CFAF
:10045000EFFFF32A0A0EF364E7D7F350D924E96ECD
:10046000000EDA20EA6EEF6AF3500AEE3FF0E9265A
:10047000000EEA22EF50006E00C002F0036A00EEA8
:1004800010F0D950E926DA50EA2202C0EEFF03C08C
:10049000EDFF0AEE40F0C151E926C251EA22EF50C9
:1004A000016E006A00EE10F0D950E926DA50EA2217
:1004B0000050EE260150ED2200EE10F0D950E92652
:1004C000DA50EA22EE06010EED22090E006E00EE71
:1004D00010F0D950E926DA50EA22002804D0D8904A
:1004E000EC32ED52EF32E82EFAD70AEE41F0C1516C
:1004F000E926C251EA22EF50006E00C002F0036A02
:10050000070ED89002360336E82EFBD700EE10F027
:10051000D950E926DA50EA220250EE260350ED22A5
:100520000AEE3DF0C151E926C251EA22EF50006EB9
:100530000AEE3EF0C151E926C251EA22EF50036EA5
:1005400000C002F000EE16F0D950E926DA50EA2297
:1005500002C0EEFF03C0EDFF0AEE42F0C151E926F2
:10056000C251EA22EF50006E016A026A036A080E65
:100570006BEC57F000C0C7F001C0C8F002C0C9F072
:1005800003C0CAF00AEE41F0C151E926C251EA2285
:10059000EF50006E016A026A036AC7510026C85113
:1005A0000122C9510222CA510322080E6BEC57F0F6
:1005B00000C0CBF001C0CCF002C0CDF003C0CEF043
:1005C0000AEE40F0C151E926C251EA22EF50006E16
:1005D000016A026A036ACB510026CC510122CD5137
:1005E0000222CE510322080E6BEC57F00AEE3FF0C8
:1005F000C151E926C251EA22EF500024046E000ED8
:100600000120056E000E0220066E000E0320076E0C
:1006100000EE12F0D950E926DA50EA2204C0EEFFCB
:1006200005C0EEFF06C0EEFF07C0EDFFED52ED5234
:1006300000EE0EF0D950E926DA50EA22EE6AED6AB1
:10064000010C0001C051020AD8A40AD000EE0CF03F
:10065000D950E926DA50EA22EE06000EED5A09D00A
:1006600000EE0CF0D950E926DA50EA22EE2A000E0C
:10067000ED2279C000F07AC001F000EE0CF0D95004
:10068000E926DA50EA22EECF02F0EDCF03F0015076
:10069000035C02E10050025CD8A02CD600EE10F002
:1006A000D950E926DA50EA22EE6AED6A000CBA0067
:1006B0000001BC6BBD6B000100EE16F0BA51E926DB
:1006C000BB51EA22D890BC35006EBD35016E230EB9
:1006D0000024E16E0C0E0120E26EEECFE6FFEDCFBE
:1006E000E5FFBAC0C7F0BBC0C8F021D8006E00C09B
:1006F00002F0036A03500210D8B4000C0001BC4B96
:10070000BD2B010EBD5D810ED8B4BC5DD8A0D3D782
:10071000000110EE16F0BA51E126BB51E2220FEEB5
:1007200025F0E6CFEEFFE5CFEDFF010CC700C7C017
:10073000E1FFC8C0E2FF00EE0EF0E150E926E25012
:10074000EA22EE2A000EED2221CA02F0036A00EE30
:100750000EF0E150E926E250EA22EECF00F0EDCFB4
:1007600001F0C7EC56F001500010D8A4010C83C072
:10077000CBF084C0CCF085C0CDF086C0CEF000EECA
:1007800016F0E150E926E250EA22EECF00F0EDCF7C
:1007900001F001C000F0016A026A036A0001005022
:1007A000CB270150CC230250CD230350CE2300EEA3
:1007B00016F0E150E926E250EA22EECF00F0EDCF4C
:1007C00001F00050C96FCA6BE1CFC7F0E2CFC8F0AB
:1007D000D890C937CA37CBC0CFF0CCC0D0F0CDC08D
:1007E000D1F0CEC0D2F0230ED36F0A0ED46FF0EC4E
:1007F0004DF0006E00C002F0036A03500210D8B43E
:10080000000C00010AEE23F0C951E926CA51EA2280
:10081000EF50006E0AEE24F0C951E926CA51EA22CF
:10082000EF50036E00C002F000EE16F0C751E9264B
:10083000C851EA2202C0EEFF03C0EDFF010CD00058
:10084000090ED2C000F0D3C001F0D4C002F0D5C070
:1008500003F076EC57F000C0E4F001C0E5F002C010
:10086000E6F003C0E7F00001D251DC6F010ED315B2
:10087000DD6FDE6BDF6BD0C0D9FFD1C0DAFFD651A0
:10088000DC25006ED751DD21016E000EDE21026EE7
:10089000000EDF21036E000E035C08E1000E025C17
:1008A00005E1020E015C02E1000E005CD8B00BD045
:1008B000D651E06FD751E16FE26BE36BD86BD96B28
:1008C000DA6BDB6B25D0DC0EE96E000EEA6E000100
:1008D000EE500008E06F020EEE54E16F000EEE5491
:1008E000E26F000EED54E36FED52ED52D6C000F012
:1008F000D7C001F0026A036AE051005CD86FE15191
:100900000158D96FE2510258DA6FE3510358DB6F97
:100910000001D890E435006EE535016E230E002409
:10092000E16E0C0E0120E26E00EE16F0D950E926C1
:10093000DA50EA22E6CFEEFFE5CFEDFF00EE0EF053
:10094000D950E926DA50EA22E4C0EEFFE5C0EDFF17
:100950007BC0E8F07CC0E9F07DC0EAF07EC0EBF03F
:1009600021CA02F0036A00EE16F0D950E926DA50E7
:10097000EA22EECF00F0EDCF01F0FE0E0026FF0ED2
:100980000120016E4FEC57F004C000F005C001F0EB
:10099000026A036A0050E8270150E9230250EA2363
:1009A0000350EB2321CA02F0036A00EE0EF0D95087
:1009B000E926DA50EA22EECF00F0EDCF01F0C7ECE5
:1009C00056F0026A036A0050E8270150E9230250FA
:1009D000EA230350EB23D9CFD0F0DACFD1F0E8C02F
:1009E000ECF0E9C0EDF0EAC0EEF0EBC0EFF0DCC0F7
:1009F000F0F0DDC0F1F0230EF26F0A0EF36FE0C0ED
:100A0000F4F0E1C0F5F09FEC4DF0006E00C002F094
:100A1000036A03500210D8B4000C0001DB51D81156
:100A2000D911DA11D8B4010CD890E435006EE5354F
:100A3000016E250E0024E16E0C0E0120E26E00EE28
:100A400016F0D051E926D151EA22E6CFEEFFE5CFEC
:100A5000EDFFD0C0E1FFD1C0E2FFE4C000F0E5C08F
:100A600001F0E6C002F0E7C003F0002A000E012208
:100A700000EE0EF0E150E926E250EA2200C0EEFF5F
:100A800001C0EDFF7BC0E8F07CC0E9F07DC0EAF07A
:100A90007EC0EBF021CA02F0036A00EE16F0E150CE
:100AA000E926E250EA22EECF00F0EDCF01F0FE0E93
:100AB0000026FF0E0120016E4FEC57F004C000F03D
:100AC00005C001F0026A036A0050E8270150E923DB
:100AD0000250EA230350EB2321CA02F0036A00EE1E
:100AE0000EF0E150E926E250EA22EECF00F0EDCF21
:100AF00001F0C7EC56F0026A036A0050E827015083
:100B0000E9230250EA230350EB23E8C0ECF0E9C0EC
:100B1000EDF0EAC0EEF0EBC0EFF0F06BF16B240EFD
:100B2000E025F26F0A0EE121F36FD8C0F4F0D9C0CE
:100B3000F5F09FEC4DF0006E00C002F0036A035028
:100B40000210D8B4000C010CC7007BC0C9F07CC0F7
:100B5000CAF07DC0CBF07EC0CCF0C7C0E1FFC8C0FA
:100B6000E2FF21CA02F0036A00EE16F0E150E92626
:100B7000E250EA22EECF00F0EDCF01F0FE0E0026AB
:100B8000FF0E0120016E4FEC57F004C000F005C0CD
:100B900001F0026A036A00010050C9270150CA230C
:100BA0000250CB230350CC2321CA02F0036A00EE8B
:100BB0000EF0E150E926E250EA22EECF00F0EDCF50
:100BC00001F0C7EC56F0026A036A0050C9270150D1
:100BD000CA230250CB230350CC23C9C0CFF0CAC0D4
:100BE000D0F0CBC0D1F0CCC0D2F0230ED36F0A0E20
:100BF000D46FF0EC4DF0006E00C002F0036A0350B9
:100C00000210D8B4000C010CD96E15D0120EE8CF2A
:100C10001EFA010EE8CF1FFA12D00A011E53D8A403
:100C20000ED00A011F53D8B4000C1FCA00F00028D0
:100C3000D8B4000C04D0D950E9E0010AEEE000017C
:100C40008D0EC96F000ECA6F1ECACBF01FCACCF042
:100C5000CD6BCE6B010ECF6F4ED923CA1EFA24CABC
:100C60001FFA010C00018D0EC96F000ECA6F120E23
:100C7000CB6FCC6BCD6BCE6B010ECF6F3CD9F66AD0
:100C8000F76A010ED96E11D0D950120AD8B40CD01F
:100C9000D950040D230EF324E96E0A0EF420EA6EF7
:100CA000EF50F626000EF722D92A230ED964ECD78E
:100CB000F6CF00F0F7CF01F01200BA000F01346B4D
:100CC0000001C26B0001C2519FDF0009D8B40ED1F0
:100CD000010E0001C26FF46A05D1F438E846E00B5A
:100CE000020FF36EF3500AEE23F0E926000EEA221B
:100CF000EF50D8B4F6D0F3500AEE23F0E926000EF8
:100D0000EA22EF50800AD8B4ECD0F3501AEE24F067
:100D1000E126000EE222BCC0E9FFBDC0EAFFE7CF3A
:100D2000EFFFF3501AEE25F0E126000EE222BEC0DE
:100D3000E9FFBFC0EAFFE7CFEFFFF3500AEE3FF055
:100D4000E926000EEA22EF50006EF3500AEE40F062
:100D5000E926000EEA22EF50036E00C002F0C0C088
:100D6000E9FFC1C0EAFF02C0EEFF03C0EDFF020EC3
:100D7000D96ED92AD950130AD8B4010CD950000120
:100D8000BA25006E000EBB21016EFD0E0024E96E37
:100D9000FF0E0120EA6EEF50D8B411D0F350D9CF36
:100DA00000F0016A0026000E0122230E0024E96EE5
:100DB0000A0E0120EA6EEF50A00AD8B492D0D950A2
:100DC0000001BA25006E000EBB21016EFD0E00244D
:100DD000E96EFF0E0120EA6EEF50D8A411D0F35057
:100DE000D9CF00F0016A0026000E0122230E002454
:100DF000E96E0A0E0120EA6EEF50A00AD8A471D065
:100E0000D9500001BA25006E000EBB21016EFD0E07
:100E10000024E96EFF0E0120EA6EEF50D8A411D035
:100E2000F350D9CF00F0016A0026000E0122230EF4
:100E30000024E96E0A0E0120EA6EEF50A00AD8B431
:100E4000010CD9500001BA25006E000EBB21016EC5
:100E5000FD0E0024E96EFF0E0120EA6EEF503F0AFE
:100E6000D8A40FD0F350D9CF00F0016A0026000EAD
:100E70000122230E0024E96E0A0E0120EA6E3F0EC5
:100E8000EF6ED9500001BA25006E000EBB21016E35
:100E9000FD0E0024E96EFF0E0120EA6EEF502A0AD3
:100EA000D8B4010CD950BA25006E000EBB21016EDA
:100EB000FD0E0024E96EFF0E0120EA6EEF50006E79
:100EC000F350D9CF02F0036A0226000E0322230E4C
:100ED0000224E96E0A0E0320EA6EEF500018D8B41F
:100EE00048D7F42A070EF464F8D6ECD63E0EE8CFC5
:100EF00034FF000CC900CBC02CFFCCC02BFF046A10
:100F0000056A066A076A0001CB07CB29D8B41CD052
:100F1000CBC000F0016A00503D0FF66E0150F76E35
:100F2000120EF7220800F550016E006A000E01BE95
:100F3000FF0E026E036E005004260150052202507F
:100F4000062203500722DFD70001CC51016E006A50
:100F5000000E01BEFF0E026E036E0050042601500B
:100F600005220250062203500722CD510426010E0D
:100F7000D8B00526D8B00626D8B00726C9C0D0F00C
:100F8000CAC0D1F004C0D2F005C0D3F006C0D4F07E
:100F900007C0D5F0CEC0D6F0CFC0D7F020EC04F01B
:100FA000010C006E046AD890FD0E01241AE3036A56
:100FB000F00E011403E1040E036E013A026AD890A8
:100FC000032A0136FDE301320150005CD8B0006E07
:100FD0000236032EF8D704BE026C025004BE006C29
:100FE0001200013206E20132D8A0006AD890003225
:100FF000D8A0D89000C002F0006A0036ECD7FFFFFE
:101000000D0A43494428303929205B70726F646EA1
:10101000616D655D203D2025303258000D0A434941
:101020004428303829205B70726F646E616D655D95
:10103000203D2025303258000D0A434944283037DE
:1010400029205B70726F646E616D655D203D2025A7
:10105000303258000D0A43494428303629205B704D
:10106000726F646E616D655D203D202530325800E1
:101070000D0A43494428303529205B70726F646E35
:10108000616D655D203D2025303258000D0A4349D1
:101090004428303429205B70726F646E616D655D29
:1010A000203D2025303258000D0A43494428313074
:1010B00029205B70726F646E616D655D203D202537
:1010C000303258000D0A43494428313529205B301D
:1010D00078204D6F2C59655D203D20253032580019
:1010E0000D0A43494428313129205B307820485784
:1010F0002C46575D203D2025303258000D0A4349CB
:101100004428303329205B6D616E75662D49445D3E
:10111000203D2025303258000D0A43494428303202
:1011200029205B6D616E75662D49445D203D20254B
:10113000303258000D0A43494428303129205B6D74
:10114000616E75662D49445D203D20253032580082
:101150000D0A43494428313629205B372D31203D83
:101160004352435D203D2025303258000D0A43494B
:101170004428313429205B73657269616C20235DDA
:10118000203D2025303258000D0A43494428313390
:1011900029205B73657269616C20235D203D2025E9
:1011A000303258000D0A43494428313229205B73FC
:1011B000657269616C20235D203D20253032580026
:1011C0000D0A435344282530326429203D20253020
:1011D0003258000D0A0D0A43534420726567697343
:1011E00074657273202831366279746573290D0A2B
:1011F0002D2D2D2D2D2D2D2D2D2D2D2D2D2D2D2D1F
:101200002D2D2D2D2D2D2D000D0A0D0A4349442085
:1012100072656769737465727320283136627974F8
:101220006573290D0A2D2D2D2D2D2D2D2D2D2D2DB7
:101230002D2D2D2D2D2D2D2D2D2D2D2D0000151568
:101240001515151515151515151515151515151350
:10125000131313131313121212121212111111116C
:1012600011111111111100FE81FE0000FEC1FE00DE
:1012700000FEE1FE0000FEF1FE0000FEF9FE0000AF
:10128000FEFDFE0000FEFFFE00181FC1F808184218
:101290003C817E322AE72A32E251E26492F591657E
:1012A00061955C6202625CFA00F090FE3E3E363E62
:1012B0003E384444282800FE7C381010387CFE005C
:1012C00060FFF9DF600C1FFC1F0C88CCEECC88227D
:1012D00066EE6622387C7C7C382070A8203E0804AC
:1012E000FE04082040FE40201010543810103854DE
:1012F0001010808894A28080A294888040707C70B6
:1013000040041C7C1C0400000000000000BE000023
:10131000000E000E0028FE28FE284854FE542446E5
:101320002610C8C46C92AA44A000000A0600003827
:10133000448200008244380028107C102810107C61
:10134000101000A0600000101010101000C0C000AD
:101350000040201008047CA2928A7C0084FE800059
:1013600084C2A2928C42828A9662302824FE204E49
:101370008A8A8A7278949292600602E2120E6C92C5
:1013800092926C0C9292523C00CCCC000000AC6C5F
:101390000000102844820028282828280082442899
:1013A000100402A2120C6492F2827CF8242224F827
:1013B000FE9292926C7C82828244FE82824438FE4B
:1013C00092929282FE121212027C829292F4FE108B
:1013D0001010FE0082FE82004080827E02FE1028F5
:1013E0004482FE80808080FE041804FEFE081020E7
:1013F000FE7C8282827CFE1212120C7C82A242BC93
:10140000FE1232528C4C929292640202FE02027ED2
:101410008080807E3E4080403EFE403040FEC628B8
:101420001028C60E10E0100EC2A2928A8600FE821C
:1014300082000408102040008282FE00080402049A
:10144000088080808080000204080040A8A8A8F0DE
:10145000FE90888870708888884070888890FE70B8
:10146000A8A8A83010FC12020410A8A8A878FE10A2
:101470000808F00090FA80004080887A0000FE2082
:1014800050880082FE8000F808F008F8F81008087C
:10149000F07088888870F82828281008141418FC20
:1014A000F81008081090A8A8A840087E8880407806
:1014B000808040F83840804038788060807888505C
:1014C00020508818A0A0A07888C8A8988800106C20
:1014D00082000000FE000000826C1000040204087C
:1014E00004F0888488F00000000000FEFF33FFFE57
:1014F000FFFFDBFF767EFFC3C3C3FFFFC3FF7EFF9B
:10150000FFDBDBC3FFFF1B1B037EFFD3F776FFFF71
:1015100018FFFF00FFFFFF0060E0C0FF7FFFFF3C00
:10152000F7E3FFFFC0C0C0FF071C07FFFF3F7EFCC3
:10153000FF7EFFC3FF7EFFFF333F1E7EFFE37FBEC4
:10154000FFFF3BEFC6CEDFDBFB7303FFFFFF037F35
:10155000FFC0FF7F3F7FE07F3FFFE038E0FFC7FF36
:1015600038FFC70F1FF01F0FE3F3DBCFC7000000EA
:10157000000000000000000000000000000000006B
:10158000000000000000000000000000000000005B
:10159000000000000000000000000000000000004B
:1015A000000000000000000000000000000000003B
:1015B000000000000000000000000000000000002B
:1015C000000000000000000000000000000000001B
:1015D000000000000000000000000000000000000B
:1015E00000000000000000000000000000000000FB
:1015F00000000000000000000000000000000000EB
:1016000000000000000000000000000000000000DA
:1016100000000000000000000000000000000000CA
:1016200000000000000000000000000000000000BA
:1016300000000000000000000000000000000000AA
:10164000000000000000000000000000000000009A
:10165000000000000000000000000000000000008A
:10166000000000000000000000000000000000007A
:10167000000000000000000000000000000000006A
:10168000000000000000000000000000000000005A
:10169000000000000000000000000000000000004A
:1016A000000000000000000000000000000000003A
:1016B000000000000000000000000000000000002A
:1016C000000000000000000000000000000000001A
:1016D000000000000000000000000000000000000A
:1016E00000000000000000000000000000000000FA
:1016F00000000004545014440000000000000000EA
:10170000000010221022101022202210202220225D
:1017100020402220224000000000000000000000C5
:1017200000000000000000000000000000000000B9
:1017300000000000000000000000000000000000A9
:10174000000000FE7BFF7BFEFE7AFE7AFEFC78FC4A
:1017500078FCF878F878F8F070F070F0E060E0600D
:10176000E0C040C040C000E020A0A0A020A0A0A0F9
:1017700020A0A040800000000000000000FCFC044D
:10178000048404F4946404F4A4E4047444F4440469
:1017900004FCFC00000010F01000F0501000E010FD
:1017A00010000000000000000000000000808080A9
:1017B0008080800000000000000000FF0043300B2C
:1017C000005B6803784B320000FF002020A87020E7
:1017D00000FEFFFEFEFEFEFEFEFECE868686CEFEEE
:1017E000FEFEFEFEFEFFFE0070887101F900F901A9
:1017F000F90070897100F8002020A8702000F8FE20
:10180000FF8F070303070707D8D8D8D88800001F21
:10181000101E101E101E101E101E101E101F000085
:1018200000000000007F7F7F7F7F7F7F7F7F7F7F43
:10183000437F7F7F7F7F7F7F7F7F7F00000000006F
:101840000000000000000000000000000000000098
:1018500000000003070F0F0E0E0F0F07000000001F
:101860000000D0D0D0D0D0D0D0D0D0D0D0D0D0D018
:10187000D0D0D0D0D0D000E0B010F000F010D050D8
:1018800050700080E010F0000000E0B010F00000A8
:1018900000000070D010D050D010D050D010D070B8
:1018A0000000D0D0D0D0D0D0D0D0D0D0D0D0D0D0D8
:1018B000D0D0D0D0D0D0EEEEEEEEEEEEEEEEEEEEFC
:1018C000EEEEEEEEEEEEEEEEEEEE0000FF80FF004E
:1018D0007794A5BD837E003F202FE984EC1800FF9C
:1018E00080FF000E0A0A0EE0BF80BFA0BF80BFA02D
:1018F000BF80BFE00000EEEEEEEEEEEEEEEEEEEEBE
:10190000EEEEEEEEEEEEEEEEEEEEFDFDFDFDFDFD9D
:10191000FDFDFDFDFDFDFDFDFDFDFDFDFDFD0000F1
:101920007C50200C503C00000020403C0040007CDB
:101930004438007C54007C14680038443800384433
:101940005434007C54007C540000FDFDFDFDFDFD81
:10195000FDFDFDFDFDFDFDFDFDFDFDFDFDFD8884A5
:10196000817F807D767A7F7D807F807F7D7C7F8494
:1019700085817D81857F777B7A777B7D7D868D8D67
:10198000888081817C7B7A7C7B807D808885818852
:1019900088807C7C818585848581817C7272787A5F
:1019A00078787F85888685898983857C77817D7A2B
:1019B000817D7B80807C7B808381838385817D7C2E
:1019C0007B7C7F7B7A7C85928F80888A7D7B7B7312
:1019D000767C7D7C8381808183848180817F858A00
:1019E000857D7F81857D73788376738084868B8BFC
:1019F0008A8E89817D8181807C7B78787D7B7B83E9
:101A000081888E7F7A847B7684817B837C7A8990BF
:101A10008D888A8684867D7A7B807D7D8B83858F89
:101A2000817C868377848A85928A7B7A807D7A76A8
:101A30007B7D77767F8B8E88868F8A8B8F7D7B816F
:101A40007B7A8083858E8673777C8889888E867B77
:101A50007178857C737684888F988E8D8475787A7A
:101A60007C7D88888588857B706B7076787680929F
:101A70008D8581767A837B8190867B7F7A7F859046
:101A8000908A92898686726C757A778597978B8013
:101A9000807D8E8B92988A81776B717269707D815F
:101AA000787D89847D7A7B7C7F929E9E8E858184E1
:101AB0007A818E8B8E786E7D7D787380817B7D7C44
:101AC00078665E666E76939A958A83757A8A7F7D4C
:101AD0009393857D86776E7B8A857C898D838378D9
:101AE00086979A8F99978D7C71777C6D83978068A4
:101AF0006E717375778F948D837D8385728E9F8DC4
:101B00009490756758687F6862787B6766757C819A
:101B100092A3A1988072767776909F9A88908A6D2A
:101B20005D6E8E978BB1A3837D6E7677787A8B907E
:101B3000765561636466979E8A898D85686C8B9EF5
:101B4000907C9C97888A8389909F958A7D6E6C7F14
:101B5000786D7588806E838F8172737A7A63737AF9
:101B60007C94A4A28E83686C8080939E8D767F8BFC
:101B70007B8999B8BDA7907A76615A6C778D856814
:101B80005E625E617183A1B3A98A847F7B8AA19D15
:101B9000988D817B6E554E63616C8D928F787169E3
:101BA000677284817394957C788F909EABB0A98A7C
:101BB00069625C6C857D8DA49E77777F6B76A3AC24
:101BC000BA975A3F4E68688394757685767A7A9389
:101BD000C2BCA88B665D7288A4A4ABA2A69F8A85AE
:101BE0008B979A997F4B313941576C696B716B8038
:101BF0009D9497B0C79D716B554B698390ADB3971A
:101C00007CA897B0CEBC936B533B44536B939D978A
:101C10008372555D8FB2B0957270858B9992817188
:101C20007C837B73678EB2B0A8734F3B3F72838017
:101C300078817A554B4F63AED5D1C58D58576668BC
:101C40007081754F595D629ACFC5E4D8B28D8178A5
:101C50006E69666B6B64667D9CA89CAD975D5267F0
:101C60005A6677687A9D86718EB8C9DDE0D3B89DD3
:101C7000888668522C3C5F7C9A89617D675F615FD2
:101C8000585F8E9E97806771787C868095B2A78D0D
:101C9000816B709EC1DDD0AC86816B4F7680788978
:101CA0007564728BA2A1AC9877635A4136437395E1
:101CB0009CA2B0A195839092818D8F71685A6E819C
:101CC000B5CA986B6363818E978D978A76676968CA
:101CD00098B6BBB69D69403B41445E85B8D3C4AE5F
:101CE0008F626B8A97A197A8A88150464844679F46
:101CF000A1978A7A6E737D8D8D9C7B706462769ECF
:101D00009EA6AE9594998A847371676C55413B5039
:101D100073858090928D8A868B909CA685523F35E4
:101D200045647F9D9A90CACCD0C6B6A3A699776425
:101D30005E4F6684AEAB9F959A8D9A8D70625A40C5
:101D400032272A3F6997B7C59E837B76626E9A8F4A
:101D50009C9F81768DA7B2BBBC938E947D686D7C71
:101D60008576897D6D6D988D7A9E945A4F575586EC
:101D7000BCD3D9C18A67433441625F7D7A7C707F6E
:101D80008BA9C9D6AE7B492B2B445D92BAD1CEBF6D
:101D90008F7D6C4A4B5D443F414A6EBADDD9D4C653
:101DA000A3774F313A5064718486735F677F728581
:101DB00093A890624D44434581B6C6D4D4C7B19C24
:101DC0009AA89F8BA6A9A8A7AE897F5A4F524A37D7
:101DD0003C64725D6278807C7B675C434139437B05
:101DE0009AC1D5DDE0C9B6A19C9A8980644F52772B
:101DF00072889475698D97888A956669677B6E8904
:101E00009A9D9592897277A9BFADA6A489685A2B2D
:101E1000172C4A73ABC9BCB6A77F5A7390A389939A
:101E20009249354157759E90736241313E5C7F9572
:101E30009A696C9D9A7694AC8A77695E5569838AB3
:101E400083958B6457617375665A585A89A6D0F783
:101E5000F8F1E0AD848B8698BCC0A190715A778967
:101E60008F9E784E4913164A7DBCDAC98D3B1C1DE6
:101E70002C4EA6D0B8BCA48F7B6E7C958F868A7BB7
:101E8000587D8F889FB6BFB89F7035212D315DA2D8
:101E9000A177615A668581757A583C5E7C7197A1FD
:101EA00086808AB299A9D8BC95A78A415268547C89
:101EB000B3BAB1A37D64503E64927B59644A374EF5
:101EC0006D7C8D94758E9A6E788E867684937D84E3
:101ED0009D885A4B4E443C5E8699A8AE979CADBDFA
:101EE000A49EADC2A6907B64585F98D3E0DED49FD9
:101EF0005F432C20467C6E5339252D73CAE5E3CB16
:101F00008936222234697F9DBC8B687080A4CAC93F
:101F1000CBB7806E5A5385D3EAE4DDBB59170F194E
:101F200046A6CCBF975843452A4B8463687A6741DD
:101F300045678ADEF9F6ECC95816162A4EB6ECD17A
:101F40009C8554213F9EB0A7CACB81494A3A3B8128
:101F5000ADC7D1B0692C0F11215FB5D1BD7B4E3714
:101F6000355483979EAC81453B7198B8DACCA47BFD
:101F70005F392B344D7BCAEAF2F3D8925F645D532C
:101F80009FCBA28E88705A6C8976593F31232B32B1
:101F90004E76808EBCC7B38F7D7146497D9EB2C997
:101FA000D4CABBC6C9BF9F7D6C62504A648DB7D589
:101FB000DFD6B697611C040D182F61707798A4A422
:101FC000CFD8955C54372348A9B7C0CFCFC6B2A2AB
:101FD000A3611D1B28314E83BAC4A8A4A49D7875A3
:101FE0007A5231495A50647A7D727A8370503C43F8
:101FF000374166738BB5B6B1C6C4ADA1805A3F3BBD
:102000004A6386A7C1B7999AA88A8095958F7D97CC
:102010009EB2DACAA97A443C504550766D53647238
:1020200077535D735C3E434F556BB1E5D6C9E7DB33
:10203000B79D95684332416CA9A9B1C7BF8A75762F
:1020400084B2BDA6947A4E32447A7180A3817268BC
:102050003B1E253067B3D1DBCF9E625A464193BD0C
:102060009FAEAC7C7B949ED0DAAE9075310D21276B
:10207000256698C9DACCB89A46182F493C5E937801
:102080007276482D539DBCCEC590623A2D3C77CBDD
:10209000EAE8DEC4551D2A5578B2C7978A9E857036
:1020A000888881ABB38D8D76321E37464B69888820
:1020B000787F664A3A5F9EB0B7CFC67A3F453E3FCB
:1020C00064BAEAEFDAA86C5F647BB3C69E7C6E6488
:1020D000544E7297AECAD1AE7152435070787DA300
:1020E000996C48322C203583A39FCBC697A3B89414
:1020F00085B1B3A1835C2A1D2862AED3D8D4C0B108
:10210000ABB7A266674D2125343762887277899212
:1021100089A8A17A4519173695CBDDE7BB75504FD5
:1021200045507BB5D1CCAB75463654ABBFB3A8692F
:1021300032394658BFE7E4DEC1783B26283E614588
:1021400030343F4A61727B9AB8C0DED08F62533C14
:1021500053839ABFE3DABAB6A45F708D677276587C
:102160006B888D99B6B1A9C5C495493021193585BB
:10217000978E9FA494684148595D7AA1865C4D7200
:102180007DA2BCB6B7D5B66252483654ACC2AE8951
:1021900064718598B2C0A371846B485077818F9821
:1021A000753B3C6E6D6685814E365381B3B6C0CEAD
:1021B000B7785E69493E7BA7A79F8F635D85868A56
:1021C000A6986B5562758899A2B5A48571553F6B29
:1021D0007A583F2C232F4D769CA497756184A7B025
:1021E000BACAB68A62444469A1CACCBAAB8F6859EC
:1021F000838A6E85AB80719472547BA39D7D7386B8
:10220000714F5F624F5A76665E5E55493E6B8981BB
:10221000A6C0BCC0BAA8804D498A8E778E905D3723
:1022200066848FCADBC1A19E6E4E7BA38D927346DE
:102230003062A7A7A3A194754531496C81858F7041
:102240006972739ED1DDC4A98B5E3E355C635F7796
:102250008E75625E73887CA8C59F8072432B546420
:102260005D9CBDA6785F4F4B4D92C7AC7D5F5430EF
:102270004083A4B7D3DBBB8B7C93A4C9DBC77D4E63
:10228000443A3E78957B716D585E6C88C5D0AB78CA
:1022900068350F2B544A61644F63909CB3D1D8B01A
:1022A00061493C1D276189B2D1D5B37F71A1A69A3E
:1022B000BCB17C6D4E354A648FA1A4AC99777698F9
:1022C0009C9E9D9395928071483B4E668AA49E9CED
:1022D00083595D7376AECBAD9F8F5E32375D7D9453
:1022E000B5B2C6C4BBA87D6150404545392D506389
:1022F00077ACB2ABBC9862685E3B3B5E5A576E945B
:1023000095B1CCB0867C8389B3B5ADAD937D818F1B
:1023100094A9A8A4A184716D5F626D72735C6385DA
:10232000786257413A3A67857D6D6C63455997A647
:10233000A18689663A314E78BCD3CCB8A28B68624C
:102340008F934F498B8E70ADC7A38FA18F5A5C615D
:102350006B6B8AA289909EABA2909E9F72637A64F7
:1023600048618194A6A3937F8D9AA6B1A28158500B
:10237000576E858E8E83728A9E8B8F7C7B63302115
:10238000448184A7C09A544F4F2B548F697AB7B5B4
:10239000A89880767D8B907A685E53627583BDD4F1
:1023A000C2C5C49A6E614F35727F6272A89F868BD8
:1023B00086838383837350251925304B94ACA3A166
:1023C0009E6E55533C375C647DA2BABDA39A92754C
:1023D0007C63598677597C9D8DA2D5DECBBB9F70DF
:1023E0003E26314B80B0B5ABA4907D8AB3BA9A8BB0
:1023F0007045455370B3B5A8BDC4A69280584E49E8
:102400005280B7A795855857698AA7B19C624D4BF2
:102410005092CBBCA368391819354869816466802D
:1024200093B5C9C6CFBA977063583C32768B9AD6AB
:10243000DFCABC9C64587663456D7F5F6490B7B516
:10244000B6B8A98964523F2C284B7A93A1A1864E35
:102450003B3423366C7575AED8A99DD3B78F7C6E8F
:102460005762696B75807C728BBCD8DBD4AB723BD6
:1024700027314F7BA6CAD4B68E73838699AC9D76DE
:102480005A3E485C9ED5E2E2E2CF9E502B222F3985
:1024900073B5BABCC6B6A39D9F767171522C374FE7
:1024A00075B5DFD4BAA780452A342D324D5A708ACB
:1024B000888AA3C5C19C787F6B5E8FB8C4BA9C8B99
:1024C0006D67839A9EA17D4F2D3E558ECFDAC4C194
:1024D000AD94868D72686257648388886E5C665599
:1024E0004B6153595544506C6EBAE2B0B2984F3BB1
:1024F0004936499FA4A2C6BB887B847A90ACB79525
:10250000807D663B59849FE0F1B88E905F354D84A5
:102510008B8B9A6E434D7071C6FBF3D9D0AB7B6445
:1025200064899E767B713C39435FAEBFC4C6B0817F
:10253000685E7388705F583A4588ACC4BCA3705815
:10254000463A4F585368787FA8CCC6BFA7775E72CB
:102550007AB3BCA499907786B2BD905E362B27449F
:102560008ED3E0DDCEBD9F675371896D44523A1B17
:1025700049948BBCD3A7856D2D27352B355F6954C6
:1025800069ABCED8D0CCA869463F32406694B3D070
:10259000EDD4BFBAA1685D483A53808B98A7A39F3A
:1025A000B0C7AC73644E2D367297BCE0EAD0B694D7
:1025B0007D6B767180846671BAC0A899AB886377A9
:1025C000886B4D3A37394685C6E3E9DEB370281487
:1025D0001B345E90ACA88B6B6CA8CED0CCA44F26DD
:1025E000202054D1EFF8F3CA754F36356D8680B090
:1025F000B39E8D857672838F8B8F897A664E4481E8
:10260000B8CCCBCEA22C031322318FB58B644945B5
:10261000506490BA986C6B4E36445F92ABADB0CCC0
:10262000D5A47A7364526E9CA3A9A29A8E8D8D73E1
:1026300063758688785F737C7DB1D9B87D696634AF
:102640004194BCD6F4E9BB8971618184928A64416A
:102650004E638EB5AEA7A8713B35413E548EC1BACC
:10266000BFA7928652404A3B4B949D83ACB5A4C011
:10267000D0AD86714B2F3A4E4B64BCE8EEEEDBAE2C
:10268000724B303236527AA1BDCCCFC0BBC1A675D9
:10269000594F2D3752675F7ABFD0C0B6A35311137D
:1026A00019204976A3C2BA9D85865D558377403F40
:1026B0003F4D68A9D9E5EAE5D1B08955302A2A48C5
:1026C000739F9CB7C6B69F805C524E4B4A62898B03
:1026D0009ECCCAAB90859DA89D733B465A8EC6D5AD
:1026E000C2A978434A45559EAC80726C453262ADB2
:1026F00093536D8359548D9C6C7695857B5D485AB8
:102700008AA7D1DEC98E6666708BABAE927A7D6D7C
:102710007C9A9FB8B8783F50734D71A28F84ADB04A
:10272000C1C4AB847557545E4B3650839EB2C9C743
:10273000B18B7341231E120E14253F6CB2E7F1E9F1
:10274000C4946745283B61575DB3CFD6EEE5BAA286
:1027500071343A5D5375A7947B7A85A3A1988A5EFC
:1027600026263E83B3DBE9E4D0B897583537437863
:102770008481819785718BD1CBB6B5952D050716D0
:1027800035A1C6ADAB94684E67614E595D54637B0D
:10279000786D859CB2BBBDB28D6E7189A3C4D3D157
:1027A000C5BA8639526C48485C3434669AC0D5D56F
:1027B000C09A787A7D686D8FA69CA3A79C9CB58BE8
:1027C000626E5A1C1636372C688EA2BAB5722C224D
:1027D00018194494B7D6ECE2BC9990837578806E52
:1027E000525C778B9399AEAE9E977F553F3E326495
:1027F0009999A7C29D77938E7B8B938D8FA2936BB4
:102800007A70597B97A6B0C9BA752A4076787DBD93
:10281000AC7B6678788E8A69463B35232B49648F7A
:10282000ADBBC1BDB0979C9C92B7B29DA38D677C98
:10283000888FBBB7976E4B20274553595D5A678FDA
:102840009AA7C6D9CEBDA889705F888988858E95DC
:10285000A8BFB06C55440D1634254F7A7770888820
:10286000725762868049638A77667797ADB1D4D311
:10287000BFAE8A636770787D8190868D94816D7517
:102880006B5E4B3C59765559A4BAADCAE2D8A986BD
:102890007541264B727F9EC7C5B8A68E736D7D7B32
:1028A000665946444A73B0AB787B69281628414F75
:1028B00067807C6C739A9DB2D4DBC2C0CAC4BBA3D0
:1028C000A19DABBFAC804B2C1609133E66778A7670
:1028D00077889CB6E2C299A276548FBCCBCCD0BF8D
:1028E000987F7D664D3B260D0D2D586DB8DBBF8062
:1028F00076783E2F49524E6172675A89A19AB1C9C2
:10290000CEB58672705D507CA2C6D8D6CEC59E76F6
:10291000503C4443363A5A767097C7C5ACBDB28036
:1029200052523B2852A3D4E3E4E3C0755A4F3044DB
:102930006C70595E6C7AABD1C7AD89581B0F161CF1
:10294000326C7C6681A4A69FB6DBC9A99885615EBE
:102950009EBACBE5ECDAC0A46623263921224430A6
:10296000233A7398AEE3F4C690B3BA97A6C5B79866
:1029700088836B5E86AB956B543E262861817D858E
:102980006E524443529CB3A9B7AC6B3C4553719D06
:10299000BAB18B694D465085C5D0C0C2A17163885C
:1029A0008AADD5C7947D531E1B436E866C647171CE
:1029B000678FCCCACAB594786455859FA6A49A7CC3
:1029C000596C948B8E937848375759547F845A5753
:1029D0005C4F4648628B8E6766837585B3D6E8E8A0
:1029E000DAD5C6A28A9397868B8555465A5A677C54
:1029F0005D44484F4D5264809FA19DCAD5CFD9C533
:102A0000A898ADC1B0B0AC7D3219091230484B570F
:102A100053495E94B8D0C7A9816C4944404163735F
:102A2000738AB68A50758AA3DEF1D99E5C322D3640
:102A30006DB6DEE9D6A6777383ADD0C7A6683F3101
:102A400025305D7384AD987D6E5D627AD1EDE3CA09
:102A5000B38326163044577A6E626775899FC4C166
:102A6000AE8F503435272A504952838999B3C4EA2E
:102A7000F9ECC7C4A6704B67857C89996952556982
:102A80008BADA4986B2A1D2123558F8DA7CFB072D3
:102A900094C7AE9FBAC1B39E92807D7B6393883505
:102AA0002C402113223B5898C0D8D6A9887563586A
:102AB0005F737376887D6B67758BB3D3CEAC7250C2
:102AC000495381C7D9D3B27D4F4E73B0CECFBC86A8
:102AD0003F2D395892ACA6A2834D455D7B9DC0C663
:102AE000C2BBA38890B1AC978878481C212D2828B8
:102AF000668B696E817067634D545E5278B5CED334
:102B0000C498777D7886ADB5A19798886463648012
:102B10009E976E5F3F222A6197ACC6BF9A8E8F70D8
:102B200059839E94959C8B6972A4C9BFB5A97C4FAB
:102B3000535C392B6D866C8E8F5C4A7171535D636B
:102B400050404F7B90A6C6DFDEA77273583E77A633
:102B50008F97CACEB1C0CBADA4BAB7855237232860
:102B6000689EB0A79C9776594F6B7A7AA9B3775530
:102B7000685E77A4A9A197816E6E7C788A836D7850
:102B80006D4F313C37376E6E6184926E76A9B3A17A
:102B9000A1A37B505C7578A8DADBC6998981697A34
:102BA0009C8B70664A302D63997F98B06C312537C5
:102BB0004A72BFD5CECCBFACAEB3AEA6B19D6D440C
:102BC00032395A80ADAD8B665A81623664724D706F
:102BD00088715E7171587C9D7D647884615C615FF1
:102BE0007BA6C9D49F6461554D84A6C5CFD8D5BDF9
:102BF000A79F999780615534212D3F72A3C2D1CCF4
:102C0000C0A38478708BB79493B0925D627F667333
:102C1000AD7C4E5D4F232F86A77F706B2B1B2A3C0C
:102C20006B95ABC9CCBFD5DEC7B3B8A980788A7B1A
:102C3000839781767583848169442B25272B498668
:102C40008684B6B084B7C18D9FC7A494B0AD939469
:102C5000AB90788B5E231D203A4328356E5968C9A6
:102C6000CFB5B58B554F5566615C7A7363647290CE
:102C70008F73777861758389B6BAB0C9CFC7C1BD84
:102C8000955E445D6E8BA9C4B07D52464B3F417149
:102C90008F76668BAC9AB8EEEEDBCFB0643B4158D2
:102CA000528899726E6931194A5046769C75584F10
:102CB00063788193AEA68870647F9FB5CED5CBBA7A
:102CC0009069414F7D7C769884482B3246537FD162
:102CD000C5855446302C50A3D8D9B899A19485CA3B
:102CE000D9C6B2A8893B213445577CABBDBD9E7582
:102CF00046231D316D8BAEB388534F72999EA6A6A5
:102D0000782F1E313B4D98D1C9ABBABC8E69857BFB
:102D10007F867292BD8A718A764E628B8EA39A7379
:102D2000543C456E9EC9E0ECEAD5B2928B908E93EE
:102D30008B70716C4E5C8A958869595927091D3CC6
:102D40003E53949A718FABA1987F716876708EBA5A
:102D5000A18FB2B3A2ABA79C704B495D63719FA6D4
:102D60007A5A677B8B7F818A533B4F6192BFC9D36D
:102D7000DAD3B0B3A3719A9C4D375A5A5E92B8B267
:102D8000A38F6B553636343B414B696C4D5383856D
:102D900086A2B1AE8D5750785D4589BB858DA881DF
:102DA0006199CACEDAE2C69E78463A405278A89433
:102DB0006B6E7A7083A6A89F906C7D978B8FA4A66C
:102DC000A1C7D1AD9AAD9550679A85647771532CA0
:102DD00013172021305E8E93ACC5C7B2BBD0C0B7ED
:102DE0009D704A211E4E94B1E0EAC68B8A6B4F5803
:102DF0005054361E406B5E76CEC2A9D8C089755C31
:102E0000354683A8BDDDDBAB6B848A6D90C08D55E4
:102E1000627D90A6CECBB1854817080411365A8F33
:102E2000ACA4ACBD9E7892632631321E2B5F9ABD56
:102E3000D4DFE2CCA39E855D50443E4471AED1E028
:102E4000F3DD98635C49484A5C5D628DA7BFEAEC9C
:102E5000D9C6C18D77A78177B0905D7DA17F615381
:102E6000402B282B2B3A50496C9CA6BAB790645D36
:102E700073A1A9BACEBD8F889A97A6AB86907C3FE6
:102E8000304E525085B0B2C9C49266524159A6CB59
:102E9000CEDEB35A374E5C83C5C9A8A28183A3B2E4
:102EA000B5B2A390784A2F2F3040739AC1D3B28124
:102EB000501D121E464A677D5753839395A4A88AD6
:102EC00092765C5E685C81B29A8DD5D4A38E8A546A
:102ED00039467C696BAC9089BDC49F909D80636EC0
:102EE000778597BBC9CCDBD9C7C4B57D554D322B8F
:102EF000362F34678DCCCB9F937C3B1C2C3C304FC2
:102F00008488A1D8C79AAEB26C77A27B71814D3903
:102F10005E98A6B1AC9D805C505862777CA6BF9E3F
:102F200090713E55897C85D0BD6E54777A86D0E30A
:102F3000D3B8AB8E7171908E735D686E53587B8081
:102F4000858564463B270F0D2044497BCAA97080C4
:102F50009E8F949C8059405A8E768DAC897BA9BBFC
:102F6000AB9989412F5C909CB1C4A952315F8B9C75
:102F7000C1ECE4BBBAD1B386865E3646615E789A10
:102F8000A2BFC7B1A186694F2F37544B3A343C6179
:102F90005C62CADD9E8FA7613B7D9585A6AC7A5F9A
:102FA000577375719AADA7A29989675361707DA80F
:102FB000AD6748645D5578928FADC0C1C9AD7D7372
:102FC0004F354058638BC5CFCAC6BDC5BCB09A6EDD
:102FD000300C05173E8DA794A7A64D14284A357FBF
:102FE000B77F4B4B3B4485ADC9C58D4030323B7CF0
:102FF000D8EACFB5A2684E636C64626B8499A49DD5
:1030000099ADC2B383839D6E456B8B7C8ED5DDC934
:10301000D3C9A888766835213C697799A2725C503B
:10302000404E706168776885A4ABA8A4A98E6B66D2
:10303000694F3A525E64ACD8BC98766B6167BABD92
:10304000997557413664B1C6CFCEB672432C2F3630
:10305000578BA4BBDDCBA69DA8A2979AA89F7A52B6
:103060006E886E789292695D4E352B263C5E85C2E5
:10307000D0A15E39171C5E94A6AC75373F6790A748
:10308000B6C08F4D2B305EB0D8D8CE97492C4A723F
:103090008889AED8BD909A937AACD9D1A28A713E74
:1030A0002D6B94ABBCC1C4A1845C5D7C77624A3556
:1030B0002832446D9DC6CBBDB1A47039375D707A9E
:1030C0009E95676373697DB2C7B69E85533F415C29
:1030D000A1BDB8A97B5E59637C989F998B767B9C38
:1030E0009A8D8A8F7A597294857D7B715367B8CE99
:1030F000C5C6C199635563726E696757464A667B58
:1031000089A6BAB28A523F2B20256298A6B6C19EE4
:1031100069707C6B86A68E5C4E5F49498094AEC117
:10312000D0C18D4F3F487DB8D3C7B78053587798EB
:10313000C2D6CBB1864B404F6EA2BAB3A68E9DB01D
:103140007C4B53534E52596C5A3959818F959EA3DB
:103150008E66626E8FA8CCCCA46C45544F5A77888B
:1031600077646E9CC1CEC1BC924B35363A76BAB507
:1031700098A19D706DC1E3C1928F672A30869D9999
:10318000BDC6977559618FA3A9B08E592C34586666
:1031900068989764484034345CA3BCAD997D584925
:1031A0006C8F9494976D443C506E86ADD3B79877EE
:1031B0006C6E7173898681A1B5AD9CA3938199A42E
:1031C000ABA69F76676E787C9DBCBB9F643E5461C6
:1031D00081B1CCBB8B6967684E53757D83758380E5
:1031E000525A8F8569788669546C777F9CC7C5BCB5
:1031F00097593B445999B0AEA372414D7FB0C6C4B4
:10320000BA8A4323315D6C8DB19770637199D1E0B7
:10321000D3B57B4F322C4E90A3C7D6BDB5AC776DDE
:1032200069432A34312A4B78788AB5A1897F6B6645
:103230006C5D868059677F616899947788858B8FEC
:1032400095ACA785645F5D46579EBAB3CEC1A7997A
:103250009CA7A69C90777078888193A881718181C2
:10326000849CB2A97D626673533F717139486B7358
:1032700080A6BAC4A67D5C4D3F557672625C4B3A1F
:103280004F6B86A9CBC08B5E64545085AD92718321
:103290006C6CB2D1CEC9AB724F303B6B7171927B0B
:1032A0005866A2B7B8D0CA925F4A324698C1D1C216
:1032B000AB7827265F7CA3C4B07031181B2649ADBC
:1032C000D1AC816746395893A8BDBC80484E524462
:1032D0007FB8B09E80817F667188706681898F9487
:1032E000A4AB8E6B808E9FC0C9BCB2A671364A63F8
:1032F0004E719A94887D57556C76A9C7A87B5A342D
:10330000235392B0D0C584595D39307094897D7C47
:10331000675E595E777F685E7A7D84929DA1B1B5C4
:10332000A89976444E5E7D8F909080728BADB2B23C
:10333000A2764A4B544F69A9B197AEAB8377A7A247
:10334000A2B08E66534149678198939495724A3C26
:10335000463C35506E5C525F7B9D97A3B793666782
:10336000626E595E949A8585A18B7D9F957866469D
:103370006D6E6BB3B19DAB8B99C1B2B1C1BC8A49C3
:1033800045585571BABC92736E533B50777A75A706
:10339000D3B0858BA498909F905341392C4952719A
:1033A000A9BAB69F76452C2F4B716D7C8D8093A169
:1033B000A6B3B6ADB7C19D55495F4E5DA4A764588D
:1033C0008A8D90988670533C6D715EA3CCC6AD9E7D
:1033D0008F736371857C7578617DB39885AB9869CF
:1033E0004F35140D1D5280ABBCAB98937C7D72366B
:1033F0003163635995946195DABD9A8D6344303F8A
:103400006D7388C5DFD8BBA69A959A8B90723749A1
:103410006C89D1D9C6CBB88F754B3535558199A8F4
:10342000BAC1AC9FA2774E4B45445D6270717090FB
:10343000988D837B7F6C3C40634E68C1E2DAC69D09
:103440006636181732526CADB8A298869CB7B6CFC4
:10345000B3612C2A32529CD1DDDFD3CBA1552D2074
:10346000203B89C4AC94A3ACB6C5BCAE864B2C2A19
:1034700036499ED4C6AD9E73261D4445313F40312A
:10348000407BAED0DFD8B7975834436C859ED1BF10
:103490009EA8A97D778B6857677157406490BAE3FF
:1034A000DBC9C1A68E8E814D52A2A8A9DEDBB284F3
:1034B0007D5F160E2D3F55A1C1A39AB6B19CA69F64
:1034C0008A571C172528498DB8DDDDBF9363311D50
:1034D0001E2A58B2B698938562539CDABFC2CBA914
:1034E0006E5A6C6D757C8D927A635E6B808EB2C9FC
:1034F000B7A6A98A6781908199BBBCB18A61482629
:103500002F75A3ACB2AB8D736E5E4A3E232F34256C
:103510004A535298D6DBC4B6A87C4B3B4E624E69E8
:1035200098838FC2B898BAD5C29485693E305472D8
:1035300088A4C0D0D0C1C1C0AE938D835E34455045
:103540004375ABAB9FA1927A7389A4B097977F4ED6
:103550003F4E494F727544485D687CA3C2B68D5496
:10356000354B5D6EBAC195869F785C88A89EA6B7DC
:1035700097705F7B939ABAAD775032325D81A1D05C
:10358000D8B19F997F68707B857555596777A1B1D0
:10359000BFC6BD949EAB75372B3A2839909C6761A6
:1035A0008A7C73B8C07F4E704F324F88756B94849D
:1035B000789CBCC4C2BD8541314471A7C1BA9D800D
:1035C000676B8AA6A99C8B895A487275A8D1D3CB00
:1035D000AD704D302F5E7597AD9D838F7752869E6F
:1035E00085706E532B398DA9B1D0D1A77C6D3B135B
:1035F0001B3E5F78868163839F8D8FA7AD7F494691
:103600006B705CACE9CE92AD923E4181624B6E86AE
:103610007CB5BD8D93B1B59DA1842A0F2534407A28
:10362000C4D6CAD3C499697AACB2A48F3C130E1D18
:103630004E6490B7B6B583494A53587CAD8A5761FA
:103640004A5C9597B3D3D0C7AE774130394E5876A0
:103650009C9F8495956C738077ACD3C9B59D7B6C2A
:10366000708097A69D7A62453A4B8ECFD9D5D1B25C
:103670006C677D887B4948503544A2B2A3B7AC77CC
:10368000626E6E5E677753314B667094A78A7C7C5E
:103690007F6348434B4D72B8C2B8B29470738BA825
:1036A0009D8081623C498186A1C5B89A7F809080C7
:1036B0008595727A8D8F9FC9B78E83846449668998
:1036C000725F7F8E725E6653406281787B8B73502F
:1036D000535A4B4E7D73556E8B8BB1E7DFB39A76A1
:1036E000524A3E596E64929A8A9EB5C0C0ACB09957
:1036F0007B7B9CA79EC4C4ACB3B688534955393272
:103700005F94929DA37B53627793A29A8A6141460C
:103710005969739994694E553B31465D50487A908A
:103720007886A9B2B2C7BB99694E5D5450ABCBAB9A
:10373000B7B16D3543707397C79E5A6DB5CAD0E85F
:10374000E3B87D573B303577B8B8CAD3C2A69A9252
:103750007259362F22161C416CB0CFB7885F5C4D72
:103760003F7C946E6978817B7D98976D54525A6C3A
:103770009EC2A4787586A3B5C6D8C07C63624E503D
:1037800068767C93A3AB9EA9C4B08A9DB7A67B68DC
:103790004927214A869C9E9A937B5F6D71575241BF
:1037A0002522305A8AA9C1BCAE9EA994623F322715
:1037B000345D7D8D8D7D816E6DA7C6C4DECA956B2F
:1037C00052699EA2999D8A624F53678099C4E2E92B
:1037D000DDC19D76555E6277A29D947A4E526C78DB
:1037E0008881696655303E647C7188AB8A707383CA
:1037F000786E7F816B66573F36446C90A6B6A98879
:103800005F5053739CA299A8B08E75A6C1AE805D1F
:103810005352788BB5D6C6B5AC97692F1625496437
:1038200097A47A68989990A3A79372442831546614
:1038300098B7A68163688B9A8F6E5C5C4F678477BC
:103840006D625757708BA2BAAE9488847F6E769261
:1038500083708AB0B3AE95907D536795817B7D72FE
:103860006C7B8E9FA87C50545C688BB7D4C6ACA888
:10387000997D92AD997673542113223B5A86C7C223
:10388000A6A97C3C4D6B837A73673E344D7AB5CCE8
:10389000C7A8816758466194A383675D55548DC25C
:1038A000B7A98970736B7A9C958FB2A277706364A5
:1038B00092A89A9E8D5D44626B55648F8A88898137
:1038C00092A3ADA8A3805C4D444B5E69677A8B8A56
:1038D00083817F858EA29E7B5D4A4D4B688AB3C7EC
:1038E000B7938A704A5869715C3F3A3C4376B7C5D2
:1038F000CFD5BC97B1B198839371354B66699DC1A3
:10390000AE88717B8189A3BFAC858675768B9E76E8
:10391000575A37304B73819CAEA3867C857F6245B6
:103920003E45465E7B888D7081ADBDAC99A87A46D8
:10393000406777768F9477697B8FB3CCC7B5A195B5
:103940009490868D8A7D73736E687588838BA19E33
:1039500081616B706C8888717D582B3F81C0C7C6B0
:10396000BCA45E2143685A576E5446677F638592B4
:1039700077636E81635A716B5E7B99B1ADA297716B
:10398000585E92A3AEA69E7F8D9EAECCB586808DEE
:10399000707CA89E78697785ABBDBDBAA676553593
:1039A0005492A194815E3B32557D76738363506857
:1039B000553B44576C90B2ACA4A1907D6C66719558
:1039C000895D675A5DA6D9E7DAA683716970767D4D
:1039D000787778A9C5BFADA7905C5768788BA4A10C
:1039E0007853556988A4A99C714F463C3B69898FDF
:1039F00092886C44414D708D8A9C8449415E596D1A
:103A0000A9C6AE9878553F373C4F615F8FC4D5E962
:103A1000E9D9B8A18E695F6357596790A7B8D6D521
:103A2000CCCCC9A862403A3C5276A6C0B7A3A38BBF
:103A300075869E90775D2C1723488FA8937B5F53E4
:103A400055639E9E8A6E6673676C808466574A547F
:103A50005C6998A89E939298A9B6A88990978D972B
:103A6000959269667895B8A9A99C6C5F73778997D8
:103A70007C5F4A546C85A9B5AD926448453537449E
:103A80004F66677888838193806E81847D7C7361C3
:103A90007A999495977A483C535E719DAB989AAD0C
:103AA000A79AADA3ABB0AE997A786E6976848F860B
:103AB00089939C959AA1978F8E7B6471808BB0B50A
:103AC0009788937A64776C43373F46505C69707887
:103AD0007A72898F86858F847789938D7B6146374B
:103AE0003A547281989E97949A978AA2B3A6988E18
:103AF00080686C8F8F7B928E7B8AB0B39FB5B18FBD
:103B000083774F3C464439415D616C929580859F37
:103B10009E93867B5A32375A7D8E999F97868E98D0
:103B20009C9E9C8362574F4357819299B8BFA79739
:103B300088694D495F819DA89F89737181838BA19D
:103B400088847D7392928D95999E9D8E7D664F524D
:103B50005D6E83A39C6D758976738E95989C88683D
:103B60006769667893888893818577574943445875
:103B700073786B769299A7BAB2A69FA19C88807C35
:103B80007576726D6C787B7B8B8E75697B8D979962
:103B900094847C868F8D898E948A7866575749489D
:103BA00077938A898E90756473757592B6AD8D81A1
:103BB0007A58577A8369696B6370777B83848B8EBD
:103BC000888183786E73787171889485787367675C
:103BD0007A979E94948F89A2BCB8AE9D837B776DB3
:103BE000728385726C7D859AB6B6B5A17B544A50B6
:103BF000525567727D8E9D9D9C9C93897369674029
:103C00003B697D8EA39A8B786876889894785E5A03
:103C1000536893B3B398734F454D637A9AB1A393A6
:103C200093AECAD0CFC6B08D6B5945415E676E8BDF
:103C3000958875726C697072706861595C626E907B
:103C4000A6A9B2B2A49E8F818A7C5D546870626618
:103C5000675E677A8D988D7D7578838993A9A98F22
:103C600081929085939D93817B839CA8ABB2A98B15
:103C70007B7B73757D766D6C676992AB95889A8650
:103C80006E72808370625A5967717F8F8D85776EEF
:103C90007D7C63585C534E5F787B7A736E7D889928
:103CA000A4A397847C7B6966808A81707C858097D9
:103CB000A4A7AEA295A3A489767F7A7A8A88777022
:103CC0006C6E83897B726C5F5A6168635D5F617043
:103CD00089A3BFD5D1B598897C788A8F7859495CFA
:103CE000767B84998D7169757A888981898D8983BC
:103CF000898F887D8181859A958D978E8186808335
:103D00008E887F7B7A727177727B8B92979F9C8073
:103D1000696C6C67696C695D687B85999990897736
:103D20006B6769695F585E534B637A8183868A75D6
:103D3000758F93909A958B8F9A8B7C817C7B9390D7
:103D4000787777696471898E90A7AC998A8B909700
:103D5000978A8F908B8B94948473767C7672736C35
:103D60005F626966687C8F98989EA1A19E999094E5
:103D70007C5A6475665F70757D9CACA798775A5FB6
:103D8000665E6B7264687D89909FA1988F8D837544
:103D9000757D888D89909A94979E9A8B7C73788094
:103DA0007B70716E666769686155576C7C8A9899FB
:103DB0009E938180868581817754484E576C8D947F
:103DC00098988973717F78778E93816B6C727597F1
:103DD000BDCBBDAE9E7F67687F979EA19A8E7A818C
:103DE000A3A9ABA68B674F536B7278938F7D7B7AB9
:103DF0007B7C6C6977848E8D939077696767707C24
:103E00008085838B95909E9E886D5A5A53495E6B30
:103E10006C7A8B9797999D88696D838E8F95998B16
:103E2000838A958688948B808189898D8478766B46
:103E30005F5C69766E6B767C7C7F807B787F81901F
:103E40009D8A757A817D849D9E8A81857A6B707A40
:103E500073706E5F5F737C858F948E8486928D897C
:103E60008F908E94A8A49C9C95836D6878869EB153
:103E7000AD94888E8066647773728589807B7D7D42
:103E80007F7F766357585A6770767F8B8D8F9790B8
:103E900090999A958978737B837A6C675E525059B2
:103EA0006E817F859085757C7D7D889C95848D9ABB
:103EB0009C9CA8B6B6B0A29584767670636164586F
:103EC0005C7280858588837C7B808486787275614E
:103ED0005D6976808F8A7D7C75707B8FA1A7A790A6
:103EE0007A73666773787C787270737680A1ADABF5
:103EF000A3937C635E6D7C8B9798948B8485949F51
:103F0000988A80705A6890B0C1AE928569555363A3
:103F10007A7C777A72626E80898B7C6C553C4862C1
:103F20007C93A4A692807777767B90B0B5958388B2
:103F3000818B97A3A88567594F5876A1A698999425
:103F40007B7A8D9A978F897B6B6E7C7B7872707B86
:103F5000738BA8A8A1867B6E5C64737A7F7D777271
:103F600070717B777B7D69625C5D63687DA19D93E9
:103F70008A88898189ACC6C2B6ADA4907B78726705
:103F8000665C5D64616E7F8A92867F85837D8197A2
:103F90009086A3A8867D775757757A6B6970757C74
:103FA00095979589695C615A677D7C8BA3A3948002
:103FB000767A88837D838A81726B767D7789A9A8DA
:103FC0009C90807D8599A6A19A907F6E6977837673
:103FD000707B8871696B6B726C7288867D7C818462
:103FE0007F7B808480808480716D6C7178767C9515
:103FF00097909F977B7678857A768375738A836DA1
:1040000077868D8A9EAD90708B9A97998D856D4835
:1040100052737169808A6E718A949E94837A616109
:104020006C717B848581808578727B7B78949D8997
:10403000848D7D8386848F8170757163708E8A9084
:1040400098948F80839290868481817F86888590E2
:104050009085857A6D69615F696D6763615D616C8B
:104060006E77897363767C728EA2A3A4A8A79D97AE
:10407000938583736267616271707C959AADB6A413
:10408000A2926E6E726D70625564726E6977847AF8
:104090007A8E94A4C0BDB0A1847266757D725D5E97
:1040A0005F7586839FA781727D6D69767A8A98890C
:1040B0007C8A92847C88897F848F8A83939592A45A
:1040C0009F7D675F5263807B89998D7D888F9394F4
:1040D000888488765E5E625C6270807F7B7F838985
:1040E000847C8AACAB979C8B718177696C63555FDC
:1040F0006E787B848A8985897768615C6875808D34
:104100008588929C9780858975768F908FA8B0B0AE
:10411000B39871615F6B70897A68646C8DACAD9C8B
:104120009A947B6869726B7886867C66647F819AD4
:10413000AB856873787276818E8572789281594FDB
:1041400068758A9C978D868E9F9EA6987758666C18
:1041500069898A77A1C1A898B39F88857C67544BE9
:104160004F7F805E586B637DA2888B9581758890A8
:104170008A7062776D67705C445A666E85A4B0A1E0
:10418000A1A18D928D8181888883718BA4A4A2AE18
:10419000A190807B7A686980A8A894947B667286D7
:1041A00083887C7C817A85806C6E666771522D4530
:1041B00066697F9484858E94AEA3725872847C76EF
:1041C0006C4B4E72857C8699A9B1AEA8B6AE838140
:1041D000BBA270668471768469616E696B846D556B
:1041E0008B9A958F805C5F8594897A6861718F9FC7
:1041F0009F84696885776976675D789A8D839592E3
:104200008AABB29A9D9F808F7D4D5D86978E7A5E38
:104210004E739EB3B79867728190B3AB7F6D696937
:104220008A7655647790A39C8A7A807D90847A6B95
:104230006872735D495C7672888F6C506C8F9E9744
:104240008D948D838B9A857092A89F8A93997670AE
:10425000766853504B778F7F7A9EA3A3BAC58E8F13
:10426000A78855505E5A4E717B76666E8DBCB094B1
:104270009575619FB39EB3A48684A29E8E735F637F
:104280006B5A5971685C638AA2988D7C777B859D97
:10429000B2B190736B76777F8669555F45556978C3
:1042A0007C8386897D7FA7AD8E8D8D73688695858D
:1042B0006772A9B6A9BAAC716893978E8F7870753A
:1042C0006B808A676C8F855864806D7885867A8963
:1042D0007B71856C5367888D9A9767505E72849066
:1042E000A69A808A978F7F81899A9D7566715957A2
:1042F000998F626D816D86AEC4C6AC9A9DA7998474
:104300008F856D636D61536B8075544E555867751D
:104310008E9C8688939E9A8086837681B1A7806CD6
:104320005A6680868A777B707B9AADB2B0A7957803
:1043300066647C8D84695E5A464D756D5D45457138
:1043400094949E948688B2BFA6959370618B816980
:10435000846E535D67556C98847B8A858EB3CBC41D
:104360009E8DA79C9898715748436D9A8A7C857159
:104370005978766B706354726E667C949D928D84CE
:104380005D64869A8067625C676476836D71A6D38C
:10439000C5C1BFB0ABA1A4A78F8892B6BDA48578D4
:1043A0007F80888063584E5C6E705D6D806B646446
:1043B0005D636690AC9E998361585F554B554D5730
:1043C00077646181817B7D7C6E6B7F9FB2B0ADB184
:1043D000BABBA29E9D92A2B8AD8D94735A77767C9B
:1043E0008167677B8EA8A89F9A90775C5750484D4D
:1043F000494D55585F766E676E839294949998886C
:1044000094A18EA7B7907B9F927D93A48995B2A328
:1044100095A3886966767C88867684888493907D67
:10442000727367534F484D669A8D757F8F7B81906D
:104430008E7A887D4D436B626670725F59526698C2
:10444000B7A4979EA7A3AB9EA39283869784676227
:10445000988E779E987C9AB092899273505C5E4E4B
:104460005D7669687D7B5C728B88868F76675C453C
:1044700063BAB5857B979498A6999FB0A290988AC5
:104480006452625D6C836449739FA3ABB5B0A9AD00
:10449000A89E946C537F7C5755595E7B7B6C7681CC
:1044A0007A8E97907A665369675A5F6459697F90EC
:1044B0009099A2A48D7A8A957A7B8B7D73857D8075
:1044C000858992B2A67C8D906970886C4E5A637310
:1044D000806972949A9DADA2857C888D8B887A556F
:1044E0004E5E5740485E709CB3A1958A94B3AB90E2
:1044F0008477667B928071687A929095846E646D01
:104500007D8B7D64616B84846E8392818DA99571AE
:10451000687161495053465C8493816E68819FA3A2
:10452000ABA8927A7C9AA99A7B70716666819C8E00
:104530007584948189947D7172634D5F7769687D1C
:10454000817D808B949783706966758976626B84B0
:10455000838FA89D75758B8D7B776B5C576889976A
:1045600097A1A9AB9FACADABB8B292736C544E6837
:104570007B705F5F7290927C73787A67688369540E
:10458000555F696C7177857A7B8A6C536171676C52
:10459000736C69665777949792ABC1B08D9FA18673
:1045A00094A2765F685A576B77818E8E93B0B29FD4
:1045B0008B8488817F73646467636B6C6977887BA5
:1045C0007585806C6872717A76809C9D8164637752
:1045D000869DB0A78D7A839CAEA19AA69D8D858F6E
:1045E0008A83898F9C947C888F8E88897B68575CAE
:1045F00069625C57506E84808B897B7B7A6E6964BC
:1046000058545C58586E7D706D808A808088888090
:10461000807776959783807F70757A757B8A888995
:1046200081696C808883857D7A898F929D99857850
:10463000848F78616B6B636D6D5C636E71808B8151
:10464000808F9EA4B0A28F8E8A92A28A7186A19E2C
:104650008E8F8D7A8BAB9A9293847D907F717777D2
:104660007B84807B7A6B637D8A6C555E6C68544F6B
:1046700057585E7C86807F8594A8A1938A84808029
:1046800083787D8478757589816C696D776B6373C8
:1046900073687D83757D7F7166738888929C8D8B2E
:1046A000988E8173686C62636C77726D7B8984818C
:1046B00085817C8485808389949293857286979E78
:1046C000ADAC9DA4BCB7ADAD9C898180807A705F94
:1046D000647B7A72756B61777A6776807F86978E56
:1046E000685A6C767B858075686C7072706D7371BA
:1046F0006D7B817A89B2B1ACB0A48E8086999C8D95
:104700008080806C525C614A434D505A6776858B3D
:104710008F908E8A8E928F836870847D76706659B2
:10472000534D4E5859646D738B959497A7A99A95DC
:10473000A1AEADAEBAB29E97988E8384806C62684B
:10474000767F7D8080838686838D8D7D76837F7165
:10475000787B6B67717D807A737C99A89F8D857556
:10476000646C848D7A687689807D837A7C9A9F894F
:104770006E7080848B938E88838381807D626C854C
:1047800080705F54555D6971624F5A646C6C6D71D5
:1047900072808E8876737B817678817772819EA312
:1047A0009388909898A19781859AA199A3A38A7DCF
:1047B000807B7573635C64666C72788B8B93989264
:1047C0008A9A9C887F8F8B70626D75687585887CEE
:1047D0007D85836E7D8A7F707275787C7873818B1E
:1047E000888994938381999F9EA3A3997F778D8FC6
:1047F00077717C6C6972674D435872776D6D69662D
:104800006C738385777D8990928E858D90929C7F45
:10481000595C67616977767C8A8D9097978F7D78F0
:104820007B726D7B86887C6D696E7686897C8184DF
:104830008AA1B8B5A8A19E98867C848075696162BA
:104840005A5861707775766C666B707D8F9FA99EE4
:10485000959C9C9AACAEB2A98D7C695A6C787371A8
:104860006D6467767C7B78766E708086766D716617
:1048700059616D6966758384818E979DA1A1998622
:10488000808992958684847C858175767261556372
:10489000686E6D6D7B6D5F6C838886A1A8A8A79AF2
:1048A0009C988586888B92816C6D767383857768FA
:1048B0005F666B6B727B8188888085958F84889515
:1048C0009E9598A19D8E8385817276868D85888B35
:1048D000807A767B8A836C6361626767697580839F
:1048E000868B938A7B86989C8E78706767666E81CC
:1048F00080868589928A8A8E94989089767064667B
:104900007A7D726972807B7A777D84858E8B8181D6
:104910008697A7A1A4A4989AA295807771696D69DA
:10492000625A575A6975736E737C8697A1A3A3A6C2
:10493000A9ADA29C9783757B8076687575707D7A2A
:10494000737376756869767A78848E807673757FEE
:10495000898E887F8488857A7B7B69677A807B7281
:1049600083978E837B7870677178716E737C859086
:1049700092847B7D858B857F849098928B83807FCA
:104980007D847C7271757F807C7677787086949751
:10499000958E929493816D6C7A8076767B7F7B7D09
:1049A0008A97998F81888F908E8988898988888055
:1049B000737D83817D848472768D8B7A727A77732E
:1049C0007A7C716E8085817D8585757C857A817D17
:1049D0006B6E78717A848B8F8A726B81908B8B8EE1
:1049E0007C6C6B6C706D666370837D767D7A778688
:1049F000908B80727A8DA2A19798938989949592D1
:104A00008E8A858477666371686367625A6D8A9D52
:104A1000A9AEB3B3AEABA8A1979495907B64676938
:104A20005F5F686C6E686B77848585888589887B15
:104A30008192999994857B7C8A8D8F948F7A7885E1
:104A40007A6464716E666C726C68779095978F83E8
:104A5000767381837777858B88887F757275818B74
:104A60008375787A676B817A69666C6C6367728527
:104A70009595989E9A948A89908D85888D816B688A
:104A80007C7F7B808F94939FB0B3B5B3ACA3988A9F
:104A90007A75776D6B767676767A888D867F81806B
:104AA0007D7B776E6E676B77849089979E929394E7
:104AB0008A857A7A72645C626B777A7B73727D899D
:104AC0008E8B8F8F88889088767D84766C6B7071E2
:104AD00078848688847C7B858B857C6C5F63696B3E
:104AE000727D858D958F8F9293958F9394857C8918
:104AF000979C93939483727176817D7B81887F8468
:104B00008D8B8A857F8B8A898D978F7A777D7D7C47
:104B10007D85847D8381858D948D8476686D6D70AF
:104B2000858A847C7876777C817F7C7F858A979064
:104B3000858E8D7F818B807C817D78777A76767883
:104B40006D6664666E696973767877868F887A8811
:104B5000A29D8E8F8E807671727A7D848B898B92E6
:104B60008D7F7F8A8D848A8A867D7B8F99938F85BE
:104B70007D7B7B83868B817A84838081717A867A40
:104B8000767C8380818584868985858988807B760B
:104B90006C6E7770737A808E867C8688837B839038
:104BA00092868D8A858F8D81848F83756E6C7070EF
:104BB000707576777376837B788077808D867F813A
:104BC0007D7575868F786E787B7786867C7D8D8007
:104BD00075818F847F858D868A8A929F8D858E8A46
:104BE0008A97939492817C7B7C786C757F77767CB6
:104BF000848E8176716C707B81817871777F7D9AEC
:104C00009F99998D9095939D988A8B81808D817ABB
:104C10008081837C788A84738E85696C756B696CFE
:104C200077756D7778717372768A8A898D83847CC3
:104C30007F817D737264666C6D767B7F868A7F83ED
:104C40007C6C738886818D95937D738581767F9347
:104C5000989898999A9D929AA3978686847B7F7B51
:104C600078777F78766D69716B697A847A73818FD2
:104C7000928986837A777F8897857A8686807684FC
:104C800090867F8B857C8D9A8F899395898B88728E
:104C9000716B686C7C83736D818D8DA1A68E808F06
:104CA0008E787B776C6367767D78777C715F616CDB
:104CB0007F8D8173716B5F615E626B686B8AA4A28A
:104CC00094998B8D9CB2B1A295948E8D95928F8A7A
:104CD00085809390949E907578776C7269737B5AF7
:104CE0004F5A6C7A838A8A8D8A849D99867C726CED
:104CF00088A3ADA68F755A667C8DA4A8A497856EEF
:104D00005D4F495E6C6672889292887C7F8D889A2E
:104D10009D988E70696E7270767F76717185938EB4
:104D20007A8190806B727C786B575E4B435D737BAE
:104D30008F9C9D939AA8B2ABA6B8B69E908A806EBF
:104D4000676376807775858166585D6164777A8B55
:104D500088858B888D94867B8690928B7A6E647B17
:104D60007B90A7A19380837A72858F979F9F80768F
:104D70007C7078808F7A647F7F766B636C6B6775ED
:104D80006E665F4A5E717F90A2A9A9AEACAEA9948F
:104D90008880885746534444484F485D7892958EA2
:104DA0008E9FAB977B85948585A2A289898E838807
:104DB000A1B8BABFAE989D896E69665354675D68A5
:104DC0005E68777692A8B69D908B725A58647B86FF
:104DD000818A7D95956C637D7A6995AC8B807562CF
:104DE0005A7B7B8094887B73718495A4908F95897E
:104DF0007F7D8181665C718A888D978B7A7D768DC7
:104E000094979F92766C635F627A7C6E7373737A09
:104E10006E67677880899DB0A397817F75767D9C4A
:104E2000908A8888858E8986898688867D959376FE
:104E30005264766E7180756D676D729399959FB2AD
:104E4000C1A994A68562505053677B7A69676763EE
:104E500075ACBAB1A6A8A998898E81838D7B7C7D1B
:104E60008975707A83978EA1A89963586473777354
:104E70007673664E57647198A39EBCBBA6AD9A7AB2
:104E80005E5D535A6E806855454D49587FA6B6B051
:104E9000B2BCC6B38AA49D70596D767F6C4E4859DA
:104EA00048467D8D8399958BA7A280726E627B9315
:104EB000A29F977B686E7A999AB0AB866E77726381
:104EC00084837C7B7A7D9888838586999A97888667
:104ED000595277697597AD998984737580938D9CC4
:104EE00086738A999E9C9789928083786D777B766A
:104EF0007A81816E76626D7D94ABAC9C998F72895C
:104F00009C898176531D21304653778D9DA2A49AAA
:104F10009C9486808383724D4E4B3F406C9EA8B21A
:104F2000B3A4A8A6B0B7B8B7956762625467787A99
:104F30007B889AB2B39A8D8E887B90846253454E5B
:104F40005A85A19F92848F9399BCBAACA6765A5881
:104F50005D6678939597888A8B7661768E90B59EFC
:104F6000847F664964909FA38A817F6D5D8194836D
:104F70008B6641413E364D7B757A7F81898D786D98
:104F8000707D85816E6757544D6B8EA8A288959E63
:104F90008B8BA99986805D6D6269738D9FA8B7B868
:104FA000CAC7BCA4989F8B85665E37232D4059766F
:104FB0009D88A1B3B5B8BDBAB2B6B0A49773806EE0
:104FC0007B69818E8F8E898B696B8A8A888A9476B9
:104FD000706D868B856D6886717A7F718A75737343
:104FE00072555E6662767D948499A6AE926E9083C9
:104FF000775864583631416D697567808077887D50
:1050000086787C7885816E6C6D77768A7697B8B273
:10501000AE9CA49F9F858E9D734F5C838D887A8FF5
:105020009E90B1BBA39D97777A93806C7F77899F81
:105030008871998F787B757F7D7F77897B575E72CA
:1050400099A6958DB79D93BCAE9890896E8B81681B
:105050006C67545A55588E9D999E94938A836980A3
:10506000855D46576786805C677D57547C806B6C96
:1050700055506D4F485561625F5D739C92A7AEB00D
:10508000BAD0C1B3B89961535E677C6E64787B8592
:1050900099C4AEA2A29AA7978383866E7C6D7B8B00
:1050A000979D8F8E84869FA1859E8D636E8F9E9522
:1050B0009F7D89A69A9CA79A9392726D5A3E393128
:1050C000354B5E5A81ABA38DA7AD9AA99999856797
:1050D00044393C505F574B6D8078727A7285737A91
:1050E00088897A7066666E676885899F998D7C90DD
:1050F00090838E72625A4645688675718192A29F2E
:10510000A1C1B39DA69F957867647F9E95A7B7B709
:10511000B3AE93849D94989C90958E7A73A4A48F3B
:10512000989490978D8D997F7C6254533A2A2A3FA8
:105130005E64768A8699ADB7BAB3A2AC936D635DAF
:105140004A435866665C5A726E646E8E887B5E61F6
:105150006D544D4F63848E9799A7948A838897895D
:1051600063585E5E52505767707F809AADB8C2BD7B
:10517000B7A785636C8362616278818B97909F99F2
:10518000A3A7B2C5B38E6C7875786D7A7F889C932F
:10519000A2AEBCC6BDB8A178687753323134464E52
:1051A0006C979F9DA8BAAC9F938D785E625F5954AF
:1051B00057493B4D556C7898ADB2855E61574F535A
:1051C0004F5269635F85929897A2A8BFAE8A837F8A
:1051D0005540443A4D554D62858EA7CCDFE3BB93D5
:1051E00070757768706E9386677297A19398ABD548
:1051F000BDA195977A44484D697A5F7195988EB2B2
:10520000CEE2D5B19E9F9A7C6C4936371C203E6910
:105210007D99B3D1C4A19A8F886150635C6E61504F
:10522000464B5557769DB5A6857C867A616858644D
:105230005F4454697D83939DA89A768B81756368DA
:105240005F5467626B63788D8B97BCC29A7368807A
:10525000787172789780676E97B5A9A8BAC4AC8B3D
:105260007653504B434B6B8A8193A2BAC1CAD8DBA9
:10527000D8BFB5A39A75412A19311E2B36597A7FAA
:10528000889CB79CA28F949581625C5F4D4944587D
:105290007083858FAB897D8089959264575F575263
:1052A00046506D787186A89A8B85706D7D5F678397
:1052B0008083847D76989D989A9F9281816E8D6679
:1052C0005E64646D727A8EA99A9D8DA3A492867392
:1052D000927B6B69675F72727199ACBAADBAB6981E
:1052E000928A8A8B7675786E5F4E506878848FA824
:1052F000BCB7A6856E6D5A4A5E68768480869A90A1
:10530000847A7F848A8D7D8F7D4D485357525266B3
:1053100088908A888A7D7D7F6775775D5C5D545A49
:105320006E7D9CB8C9CCCCBDB2AD86736955534D6A
:10533000494D463F576D778BB0B5ADBFB7B5A68D1C
:105340008F836E635C555F597084909E9AA4B5AD4F
:10535000957C707D6C575872706373839297928FAF
:105360009C8A72737F7D69645D69717586A7A89F49
:105370009889999E838BA3AC9C8A8E78644B4E62ED
:105380007A808E9780856B534A554F5D7C759297D6
:105390009A9AB0AB9AA8939A90766C6C46484F490B
:1053A00064727264837F7FA49998AE9E80867778BA
:1053B000706C5F899EA2B1ABA484806B908D7D855B
:1053C000736D53645976868A98A2B2A9AD767068D7
:1053D000433A32523E46445A787FA6BDC5B3D0C642
:1053E000BCB7A99262645A614F4F5E4F57758D905A
:1053F000BCB7ACC0BC9F84765F555258687C94ABF8
:10540000A8A2A78E92989D939D7F5D544A4D5A5EA7
:1054100050696B839D8F8A7773739292858F86769E
:105420006B73718985818B8A909093928B7F757B4A
:10543000888895928A8B838598A88B724A4E3C35D2
:10544000413F53536E8AA7B7BABDB1BFB6AD8A9874
:10545000847D70373E3B44526D73819285A9C2B7FB
:10546000ACB79E8986614F5C525364808F97A6AD1E
:10547000B29E999D9C959F93686C696E6E8990858C
:10548000867F98B1B2A4816152402C313B3E354BAE
:10549000577C8F8A85A9BCBDBAC2CFB88E6E7F9269
:1054A000817D7373625D5C6970665C4F737F76713A
:1054B000708372767D9EA68A7780908E938989808C
:1054C0006D63647B8E8377868F7B7C8B8E978A80DF
:1054D0008A88695D5C648485929DB8B2B5AC97A2F8
:1054E0008466626361786C6685858893B3C0C6BC48
:1054F000B0B7A6988668504D412143442C324E6B7C
:105500007B9E8BBFC7CBD5D0C6B5A86B757C7170A1
:10551000636758645368735E7D807F777D73789985
:10552000847A7886928880758E89817D7C786C718A
:10553000667D807877737580767193999A9DA4972C
:105540007C73677C93978F9C889083767261777564
:105550007A858969708A7F86A2BBB5ABADA18D7C47
:105560008394887F714E4854535267736D77808F50
:10557000998895B3B2A3A88A63675A4F5E7F9DA7A7
:10558000908A9581708894846D574B525845557216
:1055900080806D7C98908DA2C0C0B5927B6D725555
:1055A000405C526C4D495E676263ABB6BFAC9F9D79
:1055B00098816276758B7770887B756986959E8DEC
:1055C0008594998D8F998F9A9E8A81858F898DA9CF
:1055D000A28A818192928994867666676959617000
:1055E0007A9DB0A1978E75706C717B7F8890897D54
:1055F00078786B78765E594E5D72716B807B6373E1
:10560000767B6C7386A4B0989D9D9C867B7F888AF0
:105610007881857C7A646D7C7A72727670767A771E
:105620007867686D7B88A29889B2B1AB99898978CF
:10563000807A88717A8A7566768575989C9CAD9C0F
:10564000A1939EABB59C6D7C7F7069717588988EB7
:10565000A3A4928B768B8F8A726377585F63687589
:105660007B735F675C635C72848D7A55645F5D53A6
:1056700059768B888F989C948A98A6A7A38B888349
:105680006E645D7066645D5D70716D667F899A7829
:10569000737C76868693A8B19992908A75788E9558
:1056A0009A76676C67626E7D9392899094978897DB
:1056B00099B0B7A89588816D818E9C9E9F98838EA6
:1056C000777D84999986857761506D7A80857D850F
:1056D0006D736D66756B7F716E5352484673818B27
:1056E000899F90928B779898A498887866433E5FBC
:1056F000595F64686E8185818F887D7F837B6D664D
:105700005E778A8D8F909E9889778DABA3A19D89B6
:10571000766B525E7A716B7B858A7B6E889E9784EE
:1057200099A999896D6D8F8F8A95A8B2A1898DA845
:10573000A48F94A38E807C71817B7069787A6E6966
:105740007885887A627367645A576B76737B949412
:105750007D6E838B9E9C889497867B70727D6B6632
:10576000697264636B6476756C6C8D7C7773767F1D
:105770007C81758F8D80868581807D697D7789901C
:1057800092938D8B8193807D8A8678898983938992
:10579000818A9A93939C8881837A888E777C837A96
:1057A000686E8395A4A19D9C978B9486728E867F4C
:1057B000767172766C52686D676D66536B7A78A7F6
:1057C0008F757A857864707DA6A2897B83716B6BF7
:1057D0004D52676C6E6D777B8480809F8972776C89
:1057E0005F676C859572626C7563647780A4A7951A
:1057F0009CAC937D7D7C816E73768A7A76959DA92B
:105800009F8F92A69486858B9E957F677867698324
:105810008D978E8B89907B80898D8E90846C8D8DF9
:10582000838E9490988F778F8B7F6E808684906D17
:105830005F614E4868737272677383767F95908557
:105840009983627881768B90847A63586861585D19
:10585000706E7A8564707D717FA3ABA79A869799E5
:10586000928E83847A846E757A7267708F8A7F6D68
:1058700080837A7A809077929C9C8B8899A8BAA82A
:105880009E888A80727D8A8E767672706268717860
:1058900090A8A7A29E857A7A706D78838D756E6DBB
:1058A000718690A19484888A767A766C7A72756E05
:1058B00059455C5E678B8A778E8E727B6E66847DBF
:1058C000868B6D525A6B7D8A86857B837A85837A37
:1058D0007F7B8180816D697F90998F8F7267626411
:1058E0007C848A7F8DADB5A48D8AA4C7C0B09D92FB
:1058F0008054627B7F6D5D646E7B71889298ADA4ED
:10590000A39A8467757B667C6B6B7285756B8490DC
:10591000ADB8B7ABAD9264767D8880634E49574B86
:105920005271757D7B89898972666C6C857B7C7709
:1059300070675C86959C90999D8D7D6D786D88775C
:105940006E646176687673735C646B6C8978717071
:1059500095909D9F8D9E8A94BACAB7B0AD908A7B70
:105960006E716E706E817A8D8678989D98868A7C2D
:10597000767C685E5D756E84786E80839AA2BDBA0F
:10598000B7B3ACAE9F8469665F626E677264595547
:105990005A63616B6B6B766E5D6C888F9E938E9491
:1059A00098A2ADB5A18E807B73837A6B6E5E555DD8
:1059B000676D6C5F687A8892817A7B8571708D8B58
:1059C0008A9FA286847B78848D9D9E867F8E8F950C
:1059D000A69C7B898A849384667281767876696DC9
:1059E000766D708E9EA29FA8A48A859C9C95ABAD77
:1059F0008D928B7B8684898881616B61454F617252
:105A00005972667173716B81A3A8A6979F8D677B8E
:105A10008584839A80726D6D6E6C858584757271D4
:105A20006853486E8D89979888736D5E7A9D9E7FC6
:105A3000706C6B685A5F7B88808D8D909799A7BF3B
:105A4000B09DA995836C525273807F998478727D42
:105A50007DB1C0AB9A7B81847888999C9CA79CA9D6
:105A60009E8A7380A28B7C7F8A804B415F6D7C977E
:105A7000A49F92868889979D785C506D70636C7145
:105A8000816D72898B8D857F9EBF9D72677873450E
:105A9000455C685C737C839590869EAE8E5D55599F
:105AA00072806E738B90868DABB7B0A2A49A9384EC
:105AB00072757C72483C555D727376869F9A939E90
:105AC000B3AE838194A6908890909A888E9C977AA2
:105AD000909C95958B80775C4E535D78757D7C8529
:105AE0009299929DACA89C7A6B7C8483837B7C8109
:105AF00076788B837772715E6C7C6D6C726B777C61
:105B00006C718B8383998A7094A28E80705D6462BD
:105B10005E69706D6386A1A698929399A1AB9EA3CE
:105B2000AC936B6C6B5A6B897F767A503B67847051
:105B3000715F52637C97C4BDABA8B7B7C1B69CA9CF
:105B4000AB8F76637B725853665E52578EA8A99CC2
:105B5000898B959C89948376838678858968628F02
:105B6000978F8A90949A8BA3A39D7A5D648B8E8085
:105B70008DA89A7C5F5D697D8577715343484E623D
:105B80006D765C52778F8E848D7C8F8B9AACA28FD2
:105B9000777A88785967866D6669615C859390A786
:105BA0009A8D959C94838980869CA7A19C9F9399AC
:105BB0009AB7A68A7A7D6670807C9C9F7D5D5546EB
:105BC000618389958D7368686989A49284888588C2
:105BD0009D9E88807B81887D887C7F7C8D978E923E
:105BE0007A757A7F5F70947D8E988973716D6D720E
:105BF0005F6C6C5F758D816D818B92A39A8A867BB9
:105C00006D88A6A3A79780695C787B84737C7D6888
:105C1000544F6E77A2989A957884818B8A949F8F3F
:105C2000867C776D7D717B9776665A504E6370786F
:105C300081777A8F9D93B1C09E8A89979C9EB3B6D7
:105C400098818E9C9090805F5C6269789E9C948E17
:105C50007B6663686C7B927A6C5E5A5D7B8FB1B5B4
:105C6000957C737B7D817F8E9375544B4F586E85E9
:105C7000889589727C7F6C807F69627B5D576C7BC5
:105C800072707D97A98D7B9AB6BDB7BBCCC79E803D
:105C90007B6D5759627F9A8D889C97716870687187
:105CA000898A7A71777F7699BDB09F989092909506
:105CB00099B59A89716650414D678A857568768075
:105CC0005F63817B6167706D7B88777186817C976C
:105CD00098A9A99D9C848F988F7B8D7759595F7D5A
:105CE00090A49795977364554A4A6777626D6E7270
:105CF000728381868A7572759CA199A69FA1867709
:105D0000778078899393AC9386898A7044524F57F1
:105D10005A677A80867DA1857F8590A8C1CEB3BB66
:105D2000AB907D768684755F696C769D95ADC5B5C3
:105D30007B596C5D667888977F727B807885776BFE
:105D4000838F7B7D9086867068757A73757C868A72
:105D500086767C89766E835A3A40506372718B885E
:105D60008D8D7C6D7B99A3B2BA9D7D726370868B9D
:105D700084869083869498A7B1B5A389766352648C
:105D800081817D736871929C959E957D7A717B84EB
:105D90009298938D80787D8E92A69D8F887B818648
:105DA0008B78664D4F575958646E57778990B1A9D3
:105DB000A4A7907A78899AA3A4A8868175738695FA
:105DC000998B7873685E6B6C7D787B807559586BA6
:105DD000848F9A887283714E59677C7D8F999E8FCC
:105DE00092958FA4B08D7188785C5358615F62631F
:105DF00077706D648AA19FA8B0B5A4A17F7B7C8ACF
:105E0000888D9CA19A7F7B78897F85907B7F6E713E
:105E1000758B7B7B81706E5C5C769FA1B39D767683
:105E20005D5475847A7D89858D908E94A19A9A9817
:105E3000787372555870725F5F636372685C697DD6
:105E40007C8377738178788D938D85838E9FAC90DA
:105E50008B858E8A848D808070757A8B807A80782D
:105E60007A666B66929EA3977B7575868DA18E8AE6
:105E70008E97908E92899A9493817A5E554B536255
:105E80005955575C5D7C819295A2A6998B7C888D33
:105E90008F8E9F95907F7A78776B5E6C698A998DEB
:105EA0008593978D8D888F7C7F809AA190978B8822
:105EB0008A6E4350625568767D81937D8A957B8397
:105EC000838B9A94758089765F5D61504E495783C4
:105ED0008B83777A7C7F727F99958E97A7ADB7A2D7
:105EE0009DA19075737B858B776E686B5F5258614F
:105EF0007B727599A99DA1ABA99D88737A7C7171FC
:105F00007C7884807C89897A6763697C938D938FA0
:105F10008978726169775E5D6B84737D867C80733E
:105F2000777883758384889990858DA27A76806E40
:105F30007F8B8D86886E6B676C758B8678977D7688
:105F40007B6E738A716E7F7B7D8A9A98A89489A4F0
:105F50009D8A808D808661575F6B5D556158626157
:105F60005F769598959A94A398948A97907A80836F
:105F70008F94818199846B75787075685F8386735F
:105F80007A888D8D7B7A9C98847B837B7764576637
:105F90007A6B7789897A80888D8F897D8A94938FAF
:105FA0007D89988D7D73776964646B7168575968D2
:105FB00069757B7C7676777C899099B7AD978D7A79
:105FC000777B736C66666B757A6E66726977807CB8
:105FD0009097888693908F897C768680777C84984A
:105FE0009F8F928869727C787F8D857576726157F4
:105FF0005F6D7B7C7F8875677181818F8D7C8A8FD7
:10600000717C888392998E8A7D727C8A7C787A7D75
:106010008381727F8878858D8B8686716C7C7C7C91
:1060200088786D726468716D7F858A908B7F7383C9
:10603000897C7F7B7A7764647C817C7B8898857897
:106040006C73867D7C867F7D75717C83898B8D9456
:106050008876838B93908A847C8A6E687376766761
:106060006972867786817878786E697D7172787CBE
:10607000838A8A8A9895929A938995927C8183687B
:106080006766737D71727F8E7D8081767C88777084
:10609000817B7C817F8185766E7686839A8D8998D7
:1060A000866E77847A7B7C9094887B778572757115
:1060B00067717D686268788A8A8A999E8881979ECE
:1060C0009C9A837780777271728078727A88897AE5
:1060D000848090887B717F7B615553767371688370
:1060E0008D788188ACB0A89E9495807A6B7F8B7DEB
:1060F000777C94887B7680937A6D6E77716D64750A
:106100008A8475708B8A777A8390958475706B70AA
:1061100070707F8A817A7C7B7B727A76978D889388
:1061200089887B7572838072788B887B848E979C3C
:106130008D8881766B64737B81707F8E95978B8958
:106140008E9986807669675A627578837F8697957F
:106150008F8A9C90908A7A7283807C988F8F8470CB
:10616000768180667B887F8A88807B77637773758A
:106170008D7B848E8B84868D7B7D8871697D6B6D34
:10618000807B848A8A909894888F8A8080806C70C3
:1061900068636C757F8B80848E92989298858D8BC6
:1061A00081758D7D7376767A716D6775787B777D75
:1061B0007B7C716870786E727C88998D898F9A95D6
:1061C00088807A83897384948F85838B9397859352
:1061D0008F97927A73808D6D697271645D6B808D1B
:1061E000887A8593907F7B7F8A8062717D77706CDF
:1061F00083938D787D8F929386808589665E737296
:10620000767077929889818B97928B7B839E837728
:106210008898887D6E7A907F777D928886786D8960
:106220008470738076716E719A9C938B89999C951A
:106230007C86957868778886787B8893766B707C87
:106240008E8D81779081686E8490847C7A85777753
:1062500076707A8176676472646E838084767385E3
:1062600093939C92959E978B818577716D716E6BE0
:106270006E75807D8F93898B929388817D7F8583D6
:10628000858A84818A7F787D706D7D948D84807FFE
:10629000757B787F7C807D7B8488887A8F979E95BC
:1062A000888A898E8D8F8E8B8D8389959F90838D23
:1062B0008986636E7D848D818B768B818A8E97949F
:1062C00080857F9281768180717671696B70626E54
:1062D0007573807C8B9894888D8D73736E767068DF
:1062E000646B71666B6B7888848583908880868BFD
:1062F0008B7C7A7D8A7A72727178766E7578786D19
:1063000072848B81757F8B867D7680928F80939C43
:10631000978D7D839285727A867875717293928853
:106320008F97847A6C6E8888757D9094927A6E834C
:10633000887D80858B927D778A947A777D8E857C27
:10634000757F99908E909F9E8E8989898071717BCF
:106350008B7D72768E8B8E8A909E93817A777D70FC
:1063600071768678706D7688817F848D83777A7672
:1063700085807D7B847A6C696C7A7A777A888A8367
:106380008483848472687D7C7D7575818B8486931B
:10639000929381817D8472687A7A886E717D857F1F
:1063A000849997A2938F868577717C7B897C6C72A8
:1063B000787A7F938A938F85898F8D888F908B8B46
:1063C00072767875838F8B8B8F84807B6B767673F8
:1063D0006E80726E7A778E8D958D909397988D9250
:1063E00085847D837D787D75787B81889A9E979062
:1063F000857A7B807A768176717071888E8B8F94A6
:10640000958A837A837C7C767D6E66685F69838AF1
:106410008090927F7D7F80807D6C7677676E7573CC
:10642000848A76838680868E7F85846C767C6C6891
:1064300076697F8983939C97858D819084767A8015
:1064400075677B707C7B7D848A92868F93978A8028
:10645000777B80737D84888588928D888076848E12
:10646000867B757C7A7170868583818A8F8B998D06
:106470009EA79585767673806C80857F7C809386D9
:106480008D7B888E8E7F6B6E667261788181848B46
:106490009E8F948B9494938578706371696D7073FB
:1064A000777A88857B707777807D75686661696D9E
:1064B000706E7072738378838D92979389767B6BFD
:1064C000787B807B7F8889998B94868B837B7A729B
:1064D0007A6D767580757C8881958F978F9795906A
:1064E0008D8384787D7886767881818E8D958A8A71
:1064F00088857B7B7871767385817C7C838F92998C
:10650000949495988183847C807C83887D7D8D980C
:106510009593988D7F7C7270756B5C61636D707301
:10652000838B8D8B938E8A8F8A7D7877696D6C6B68
:10653000706C6E75818090928D847B7875806770A9
:106540007C76716D7173818495949388838A7D8143
:10655000737A837A737C898A8F8B928A897C757C23
:106560007C86776E6E72616C76848B8695999A8F35
:106570008B92958F7C7A8083767F868E8D7B898EB9
:106580008D847D7A818D7B727A80777877808E801A
:106590008895998F868B9297837683867C80818B72
:1065A0009485858F8A7F757577848170767362672D
:1065B000636E85807C9299948F8B9C9A8E77757789
:1065C0006B6D6E788D8E858886847B6E76807B720F
:1065D00078786E6C6D6B777B727A808A8D8E94A3DF
:1065E000958D8D8177718077888F837D7C85838B76
:1065F0007F8D8876787569627569727D777075832D
:10660000808E8399A2938F8F7F66776E7C8A8B832F
:1066100085887C88787D8881758376677D807F8496
:1066200085767C7C7F8986889D99858B806D6C784A
:106630007C8D94898E8D888986768884737771693C
:10664000737C7B807F7A7B807F8A9495A9A79F93B8
:106650008A77757A7D7F808483858188857D7D7545
:1066600072666C5F5F6B75727577727B7775838FFF
:1066700098999E908D7B6D75757683817884837BE8
:1066800085857F80867C868A78787672837D6C7734
:106690007D7576888D979E8F8D8B7C6E76738888BE
:1066A000778088837F847F84857C7C8880767578FA
:1066B0008889787681838483949F9D958F958A833A
:1066C0007B88909084818383867F8B908B837B8370
:1066D0008077716E737C7871727C817A85908E8FF1
:1066E0008989837D78757A807F76767C77767C88D9
:1066F000817B7575787678777476726F69766A6D56
:1067000079838D8A8D888E87858583878980788037
:10671000806E78828C8C7C7D828077797E7B837B97
:106720007780807374808A948A899B9894898985FC
:10673000948E74838A80727B89918273838A807835
:10674000797D888A7C7B93877B727C888079748D45
:106750008C8080828791836A808880747485897C2C
:106760006D778A7E776E7783826B70847B6E6E74B2
:106770007E827E7E96968A887E8891797588917BC6
:1067800075727B7E70666E7C707472798983758297
:1067900090847B7C788C8C80808588877D7E8D8BB7
:1067A00080808984807E7E8385807B8083928888B8
:1067B00089908479837C7C74747B838287848890BD
:1067C0008C848B8D8984888D8789807D7B78797393
:1067D00074797E7C8288888686837E7A7C798080C4
:1067E000857B7B7E7D807D878C8C878C8F89828367
:1067F0007E807A756F787D7B807D827D77788580DD
:106800007D858B8988807C807E7E778084867C7B7A
:10681000808780747976776F6B71777D77778483E3
:106820007E777C84867D7784878980807C8480786D
:10683000808980807A7E89887D7C8680807C7C8748
:106840008B7C74867D78757980887C7484847D7C6B
:10685000787D8C867D8894888786828C8878767C03
:106860007678726D8082747580837D837E878E8357
:1068700080838C87887D838E887E7C8A807E8083DF
:1068800088867D7D7E8082807D8788807A7A827D01
:106890008383888A8383838A86837A7C807E797ADD
:1068A0008383838680837D7876797E797A767A741D
:1068B00074716F7A75787C8078807E7D8387848020
:1068C0007E8086878080858382827E7E827D7C80BA
:1068D000827E82827A827776777B7C8682808A86C5
:1068E000878A918A8E89878D8D87878C898E847C13
:1068F0007E827E7C80807D7C7B7B7E7C7A7A8085BC
:10690000847E80848282828282807B7E7E837E7A85
:106910007D87827D7A7E8280808087827E7C7A7D80
:106920007B7673807E7B7A7D8082837B85827E808E
:1069300080848782767D807A797A82827E7A807E70
:10694000767878767A7870717D7B7B7A80847E82A7
:106950008086878686868A86807D838582808085FC
:10696000807D7E797E807E8080837F807B85838032
:106970008083868390898C8B888682837F827B80CC
:1069800087868183867F82817F83807D8082807DF0
:106990007E7A807F7B7B7E808085808685808082FA
:1069A000817E7E787D82828080827F8080807F7EF3
:1069B0007B7A78777979787D7D7A7A797E7E83851E
:1069C000848182848185848681838280807D807DAC
:1069D0007D797A74757A7A7C7C8281807F80817DF2
:1069E000808487898B858282807E7F7C807A797D96
:1069F000818180868285807B787C7E777B798280AE
:106A00007A7F807E7B827F878A8A88878985898250
:106A1000888A818283868288818385807B7B7D7B57
:106A20007C787B807E787D7C7C817E808486848679
:106A3000848788848387857B7E7F7F81807E7C7B43
:106A4000767776787C7D7E82857D797B7E80848278
:106A50008285848584858785838587817B7B7C7D12
:106A6000828182807C7C7B7B7B7C7C8182807C7C45
:106A70007E7E80828682808385818385828A8A88E1
:106A80008281807E7F7E838079767C79787D7A8230
:106A900082807A7D7E7D80808685827D84838187E9
:106AA00083878B89818280808180838481787C7DCB
:106AB0007A7D7E7C80817C7D7C807E7E8084837FED
:106AC000818081808381888B84837C807E7E7E80B0
:106AD000807A7A777A777B7A7C7F7C7E7A7E7F7EFB
:106AE0007C84848282828482858384858683807F7D
:106AF000807F7A807E7F7D7C7B7C7F7F807F8382AE
:106B0000817F7F7E7C81818383828280828386866F
:106B100089888A86858480807D7D7D7C797A797973
:106B20007D7C7E7F827F80807F808182848783835B
:106B30008281838281808482807F7F7F7E7E7F824C
:106B400080807E7B7E7F7E7F82817F7D7B7B7B7B67
:106B50007D80818181808386858687878683828107
:106B600081817E7C7C7A7A79797D7D7F808181804C
:106B7000807F7D7C7F7F8182818180818182818312
:106B800085838381807E7E7D7D7B787A797B7E7F25
:106B90007F80828180807F7D7F80808181818081F4
:106BA0008485838283858281818080818180807FCA
:106BB0007F7F7E7F81817F838180807E7E80807EDB
:106BC00080818080818284837F84858384838080A8
:106BD000807C7D7C7C7C7D7C7F807D7E807F7F80D7
:106BE0007E7F818080828383858486878484868477
:106BF0008383807F807E7B7D7D7B7C7B7C7F7D7DB6
:106C00007F7F7E7F7F7F808080818281828182837F
:106C1000807E7F807F7F7D7E7C7B7C7C7E7E7F7E96
:106C20007F80807F7E7F7E7E7D7F7F7F7F7D808176
:106C3000818083848484828584848283828181802C
:106C40008081817F8081808080807F7F7F7D7F7F4A
:106C50007F8080828382838585858583838282800D
:106C600080807E807E7E7F7F7D7E80808080807F32
:106C7000807F7F807F807F7F7F8080818382828210
:106C80008180828180807F7F807F7E7F7F7D7F7F0C
:106C90007F807F7D7D7E7E7F7E7E7F7F7E7F80800A
:106CA00081818181818080808081807E7F7E7C7DEA
:106CB0007E7E7F7F7F7F7F7E7E7F808080808080E2
:106CC00080808080818282838282828281828280AF
:106CD0008080807F808080828182808080807F7FB2
:106CE000808080807F7F80808080818181818180A1
:106CF0008080818180807F7F7F7F7F7F8080807F99
:106D000080808080808080807F7F80808080818282
:106D100081808181808080818180807F7F7F7F8072
:106D20008080808080808080808080808080808063
:106D30008080808080808081808080808080808052
:106D40008080807F80808080808080808080808044
:106D5000808080807F808080808080808080808034
:106D60008080808000000000000000000000000023
:106D70000000000000000000000000000000000013
:106D80000000000000000000000000000000000003
:106D9000FE910E921E921E921E921E921E921E92A4
:106DA0001E921E921E921E921E921E921E921E9263
:106DB0001E921E921E921E922E922E922E922E9213
:106DC0002E923E924E922E923E925E926E926E92D3
:106DD0006E926E926E929C939C939C939C936E92F7
:106DE0009C939C939C939C939C939C939C939C932B
:106DF0009C939C937E928E929E929C939C939C9348
:106E00009C939C939C939C93AE92BE92CE92DE9266
:106E1000EE92FE920E931E939C939C932E933E9320
:106E20004E935E938C937D60606060606060606094
:106E300060606060607D007D53454C2E2044363498
:106E4000203A243F3F3F7D007D20313534312D49AC
:106E5000494920284A44297D007D53454C2E204332
:106E60004152443A243020207D007D44495245431C
:106E7000544F52593A242020207D00726F6F7420A5
:106E80006469726563746F7279004154413A726447
:106E90002074696D656F7574004641543A7265617E
:106EA0006420626F6F7473002573006A60606060B5
:106EB000606060606060606060606B007560606012
:106EC000606060606060606060606069004641545E
:106ED0003A6A756D70206F70636F6465004A332085
:106EE0003A20706C61636564004A32203A20706C0D
:106EF000616365640046696C653A2020253033641F
:106F00002F253033640025633D2530326420543D05
:106F10002530326420533D25303264005665723A84
:106F20002025642E253032642E25303264004452F0
:106F3000495645204E4F5420524541445900437410
:106F4000723A2030782530325800313534312D49AD
:106F500049492056005245434F5244204E4F542039
:106F600050524553454E540046494C4520455849DA
:106F700053545300494C4C4547414C2053595354AA
:106F8000454D2054204F52205300494C4C45474119
:106F90004C20545241434B20414E442053454354CE
:106FA0004F52004449524543544F52592045525282
:106FB0004F520053594E544158204552524F52009F
:106FC0005752495445204552524F52005245414470
:106FD000204552524F52004552524F5220554E4B6F
:106FE0004E4F574E0057524954452050524F54452A
:106FF0004354204F4E0046494C45204E4F54204F9D
:1070000050454E0057524954452046494C45204F63
:1070100050454E004449534B2046554C4C004E4F72
:10702000204348414E4E454C004F4B004E4F2042AE
:107030004C4F434B0046494C452054595045204D38
:1070400049534D41544348004449534B204944203F
:107050004D49534D415443480046494C4520544FF7
:107060004F204C41524745004F564552464C4F57D2
:1070700020494E205245434F52440046494C45203A
:107080004E4F5420464F554E440046494C455320E0
:10709000534352415443484544004E2F4100533A14
:1070A00000523A004E3A00433A00403A0053303A18
:1070B0000052303A004E303A0043303A0040303A05
:1070C00000434152443A65727220434D44353800C2
:1070D0004154413A6572722E20434D44313700537A
:1070E000656C656374696F6E206572722E00436112
:1070F0007264206E6F7420737570702E00556E640C
:107100006566696E65642E2E2E2E2E000D0A0D0A00
:1071100020202D2D3D3D20313534312D4949492048
:107120007625642E25642E25642C206279204A2E33
:107130004465726F676565203D3D2D2D000D0A4A3F
:10714000332028426F6F746C6F61646572293A2036
:1071500044495341424C45442020286A756D70656E
:10716000722072656D6F76656429000D0A4A3220BF
:10717000284465766963652D494429203A204944AD
:107180003A25642020202020286A756D70657220C1
:1071900072656D6F76656429000D0A4A33202842B6
:1071A0006F6F746C6F61646572293A204143544972
:1071B0005645202020286A756D70657220706C61BC
:1071C00063656429000D0A4A3220284465766963A4
:1071D000652D494429203A2049443A25642020203D
:1071E000202020286A756D70657220706C6163655F
:1071F00064290024004641543A77722E206D65645C
:1072000069756D2000204D61782E2072656163687C
:1072100065642000204D696E2E207265616368658B
:107220006420002043415244204449524543544F76
:107230005259200020464F524D415454494E472E3A
:107240002E200020205245504C4143494E472E2EBF
:107250002000202044454C4554494E472E2E2E20D8
:10726000004A33203A206F70656E2020004A322099
:107270003A206F70656E2020004641543A626C6F70
:10728000636B73697A65202000434152443A766FFC
:107290006C74616765202000202052454E414D49A5
:1072A0004E472E2E2020002020434F5059494E4754
:1072B0002E2E2E202000202020534156494E472EAE
:1072C0002E2E202000202057524954494E472E2E62
:1072D0002E20200020204C4F4144494E472E2E2E78
:1072E000202000202052454144494E472E2E2E207A
:1072F0002000496E69742E20636172643A20202058
:1073000000434152443A4F4B2020202020202000AF
:10731000424C4F434B5320465245452E20202020BF
:1073200020202020202020202020200064CFD8FFF3
:107330001000FCD7E9CF7EFFEACF7DFFE1CF7CFFD5
:10734000E2CF7BFFD9CF7AFFDACF79FF0EC078FF8B
:107350000DC077FF0CC076FF0BC075FF0AC074FF2D
:1073600009C073FF08C072FF07C071FF06C070FF3D
:1073700005C06FFF04C06EFF03C06DFF02C06CFF4D
:1073800001C06BFF00C06AFFF7CF69FFF6CF68FF4F
:10739000F5CF67FFF4CF66FFF3CF65FFF2A203D00E
:1073A000F2920FEC53F0F2A431D0D59EF29428CF94
:1073B000E8FF030AD8A420D011AA04D0119A2ACF3A
:1073C000D6FF05D0118A2ACFE8FF0008D66ED7680D
:1073D0002ACF00F00004D8B411862ACFE8FFFE0AB5
:1073E000D8B4119611A604D00F01010E2A2B08D093
:1073F0000F01010E2A0704D0117AF60ED76ED66A55
:1074000011AA02D0808201D08092D58E9EB09E902B
:1074100065CFF3FF66CFF4FF67CFF5FF68CFF6FFC8
:1074200069CFF7FF6ACF00F06BCF01F06CCF02F0AD
:107430006DCF03F06ECF04F06FCF05F070CF06F084
:1074400071CF07F072CF08F073CF09F074CF0AF054
:1074500075CF0BF076CF0CF077CF0DF078CF0EF024
:1074600079CFDAFF7ACFD9FF7BCFE2FF7CCFE1FF84
:107470007DCFEAFF7ECFE9FF7FCFFAFF1100CAEC94
:1074800055F008EC4AF0E8CF33FF33CFE8FF46EC85
:1074900051F0119000010C0EDF6F710EE06F190EAC
:1074A000A96FAA6B080EA76FA86B060EA56FA66B37
:1074B000A50EE8CFDDF0000EE8CFDEF081EC57F04E
:1074C000000182B010D0C50EDF6F710EE06F33CFB8
:1074D000A9F0AA6BA90EE8CFDDF0000EE8CFDEF030
:1074E00081EC57F00FD06B0EDF6F710EE06F33CF72
:1074F000A9F0AA6BA90EE8CFDDF0000EE8CFDEF010
:1075000081EC57F0000182B207D0990EDF6F710E47
:10751000E06F81EC57F006D03D0EDF6F710EE06F2B
:1075200081EC57F01180010E0001C96F490EC4ECC7
:1075300048F0FAEC56F012EC53F042EC53F0000134
:10754000EE0EC06F020EC16FA5EC55F00001C96BC5
:10755000490EC4EC48F00F01296B0F01306B0F018D
:10756000326B01D8FED7C80E0001CE6FCF6B66EC30
:1075700055F000012E0EBA6F0F0EBB6F010EBC6FDF
:10758000B6EC52F0E8CF31FF0F013153D8A442D00E
:107590000F0180B8296B29530001D8A432D0E80E1E
:1075A000C06F030EC16FA5EC55F00001C96B490E09
:1075B000C4EC48F02AEC53F047DB29EC3FF000091B
:1075C000D8B41ED0EFEC3FF0030E0001C96F490E96
:1075D000C4EC48F000018B6B8C6B2AEC53F08BC031
:1075E000BAF08CC0BBF00001BC6B7EEC41F0000136
:1075F000C96BCA6BCB6BCC6BCD6B000E7BEC42F0D6
:1076000000012E0EBA6F0F0EBB6F010EBC6FB6ECF1
:1076100052F0B8D7C80E0001CE6FCF6B66EC55F0B4
:1076200031CFE8FF200AD8B405D031CFE8FF400AB7
:10763000D8A40DD031CFE8FF200AD8A404D0010E81
:10764000E8CF32FF1200020EE8CF32FF12000F0126
:107650003253D8A4E4D250EF51F050EC51F00F0166
:10766000326B120050EC51F00F01326B1200F3EC50
:1076700048F0120000013B0EBA6F0F0EBB6F010EF7
:10768000BC6FBD6B72EC40F0320E0001C06FC16B7D
:10769000A5EC55F00001F30EBA6F710EBB6F3B0EF7
:1076A000BC6F0F0EBD6F010EBE6FBF6BF8EC54F0D8
:1076B000015000100001D8A48ED03C0EBA6F0F0EFE
:1076C000BB6FB40EBC6F000EBD6F95EC40F0006E4A
:1076D00000C002F0036A03500210D8B46FD000015A
:1076E000B751B411B511B611D8A40AD000018B6BF3
:1076F0008C6B010EE8CF29FF030EE8CF30FF12009C
:10770000010EE8CF29FF040EE8CF30FFB4C08BF0A4
:10771000B5C08CF00001B06BB16BB26BB36B8BC0BA
:1077200000F08CC001F0026A036A00010350B35DEF
:1077300008E10250B25D05E10150B15D02E1005087
:10774000B05DD8B034D00001B351B011B111B21155
:10775000D8A408D08D0EBE6F000EBF6FC06B5BEC5F
:1077600001F01ED000018D0EBE6F000EBF6F010E26
:10777000C06F5BEC01F0006E00C002F0036A0350C2
:107780000210D8A40DD0020E0001C96F150EC4EC72
:1077900048F000018B6B8C6B010EE8CF30FF07D0F7
:1077A0000001B02B000EB123B223B323B8D70001E0
:1077B0008D0EBA6F000EBB6F58EF03F000018B51B6
:1077C0008C11D8A404D0030EE8CF30FF1200040EB1
:1077D000E8CF30FF1200A40EBA6F700EBB6F3B0EE5
:1077E000BC6F0F0EBD6F020EBE6FBF6BF8EC54F096
:1077F00001500010D8B412000001B50EBA6F700E1F
:10780000BB6F3B0EBC6F0F0EBD6F030EBE6FBF6B29
:10781000F8EC54F001500010D8B4120000019E0E94
:10782000BA6F700EBB6F3B0EBC6F0F0EBD6F020EBA
:10783000BE6FBF6BF8EC54F001500010D8B412D0FA
:107840000001AD0EBA6F700EBB6F3B0EBC6F0F0E1A
:10785000BD6F030EBE6FBF6BF8EC54F0015000100B
:10786000D8A404D00A0EE8CF30FF12000001A10E08
:10787000BA6F700EBB6F3B0EBC6F0F0EBD6F020E6A
:10788000BE6FBF6BF8EC54F001500010D8B412007A
:107890000001B10EBA6F700EBB6F3B0EBC6F0F0EC6
:1078A000BD6F030EBE6FBF6BF8EC54F001500010BB
:1078B000D8B412000001AA0EBA6F700EBB6F3B0E57
:1078C000BC6F0F0EBD6F020EBE6FBF6BF8EC54F0B5
:1078D00001500010D8B412D00001BD0EBA6F700E66
:1078E000BB6F3B0EBC6F0F0EBD6F030EBE6FBF6B49
:1078F000F8EC54F001500010D8A404D0070EE8CFE3
:1079000030FF12000001A70EBA6F700EBB6F3B0E66
:10791000BC6F0F0EBD6F020EBE6FBF6BF8EC54F064
:10792000015000100001D8B412D0B90EBA6F700E19
:10793000BB6F3B0EBC6F0F0EBD6F030EBE6FBF6BF8
:10794000F8EC54F001500010D8A419D000013B0EFF
:10795000BA6F0F0EBB6FAD0EBC6F000EBD6FAC0EDD
:10796000BE6F000EBF6FAE0EC06F000EC16F5EEC3B
:1079700006F00001AB6F0C0EE8CF30FF12000001E3
:107980008B518C1100013B0ED8A40FD0BA6F0F0E93
:10799000BB6F8D0EBC6F000EBD6F0AEC47F000018F
:1079A000AB6F060EE8CF30FF1200BA6F0F0EBB6F41
:1079B000AD0EBC6F000EBD6FAC0EBE6F000EBF6F84
:1079C000AE0EC06F000EC16F5EEC06F00001AB6F33
:1079D000050EE8CF30FF12000F012953D8B405D0AF
:1079E00029CFE8FF020AD8A4EED032CFE8FF020A7E
:1079F000D8A404D0010EE8CF30FFE5D0020EFBD7AB
:107A000050EC51F0FFD093EC52F050EC51F0FAD022
:107A100050EC51F0F7D0010EF9DB8BC0BAF08CC0FE
:107A2000BBF00001BC6B7EEC41F065EC43F0EAD0AA
:107A3000010EECDB8BC0BAF08CC0BBF00001BC6B5C
:107A40007EEC41F08BC000F08CC001F000500001D2
:107A5000BA6F0150BB6FBC6BBD6B14EC45F0D2D05C
:107A600032CFE8FF020AD8A430D00001AB05D8A479
:107A700021D0010ECBDB020E0001D76F000E65ECAA
:107A800053F00001A80EDF6F6E0EE06F3B0EB86F73
:107A90000F0EB96FB80EE8CFDDF0000EE8CFDEF0C4
:107AA00081EC57F000018D0EBA6F000EBB6F8EECAB
:107AB00047F0A8D0020E0001C96F3E0EC4EC48F09A
:107AC00093EC52F050EC51F09DD0020E0001C96FC2
:107AD0001C0EC4EC48F0020EE8CF30FF93D032CF3A
:107AE000E8FF020AD8A433D00001AB05D8A424D003
:107AF000010E8CDB020E0001D76F000E65EC53F017
:107B00000001A80EDF6F6E0EE06F3B0EB86F0F0E18
:107B1000B96FB80EE8CFDDF0000EE8CFDEF081ECF3
:107B200057F00001AC51BA6FAEC0BBF0AFC0BCF0B3
:107B3000AD5134EC48F066D0020E0001C96F3E0E24
:107B4000C4EC48F093EC52F050EC51F05BD00001E3
:107B5000AB51020ED8A423D059DB020E0001D76F1F
:107B6000000E65EC53F00001A80EDF6F6E0EE06FA3
:107B70003B0EB86F0F0EB96FB80EE8CFDDF0000EF8
:107B8000E8CFDEF081EC57F00001AC51BA6FAEC027
:107B9000BBF0AFC0BCF0AD51B6EC48F033D0000143
:107BA000C96F3F0EC4EC48F050EC51F02BD0050EDD
:107BB0002DDB28D0030E2ADB25D0040E27DB22D0B4
:107BC000060E24DB1FD030CFE8FF000A01E118D7F2
:107BD000010A01E118D7030A01E11AD7010A01E1FC
:107BE0001AD7070A01E124D7010A01E178D7030A6D
:107BF00001E136D7010ADBE00D0ADCE0010ADDE035
:107C0000070ADEE0000E02D350EC51F0020E000134
:107C1000C96F1E0EC4EC48F00F01326B120031CF59
:107C2000E8FF3F0A01E119D5600A01E11BD53F0ACF
:107C300001E1D2D60F0A01E11AD58F0A01E119D567
:107C4000100A01E117D5E0D70001D76B000E65ECF3
:107C500053F06F0E09EC56F0010E0001D76F000EC5
:107C600065EC53F000011D0EDF6F730EE06F81ECC9
:107C700057F0020E0001D76F000E65EC53F0160EA0
:107C800009EC56F0040E0001D76F000E65EC53F0BE
:107C9000690E09EC56F00BEC4AF00009D8B412005A
:107CA00012A035D00F013507810E356118D0810E35
:107CB000E8CF35FF010E0001D76F000E65EC53F0E1
:107CC0000001140EDF6F720EE06F81EC57F00001BF
:107CD0005E0EC06F010EC16FA5EC55F018D029ECF7
:107CE00053F0010E0001D76F000E65EC53F0810ECA
:107CF0000001D76F35CFE8FFFF0844EC54F012ECD9
:107D000057F0C80E0001C06FC16BA5EC55F012A270
:107D100037D00F01352B35CF00F00028D8A418D06C
:107D2000FE0EE8CF35FF010E0001D76F000E65ECA7
:107D300053F00001050EDF6F720EE06F81EC57F01B
:107D400000015E0EC06F010EC16FA5EC55F018D09A
:107D500029EC53F0010E0001D76F000E65EC53F0D3
:107D6000810E0001D76F35CFE8FFFF0844EC54F0D7
:107D700012EC57F0C80E0001C06FC16BA5EC55F0B6
:107D800011AE89D72AEC53F00001D76B000E65ECD9
:107D900053F000011C0EDF6F6F0EE06F190EBE6F07
:107DA000BF6B080EBC6FBD6B060EBA6FBB6BBA0E15
:107DB000E8CFDDF0000EE8CFDEF081EC57F0010EE9
:107DC0000001D76F000E65EC53F000013E0EDF6F2F
:107DD0006F0EE06F35CFBEF0BF6BBE0EE8CFDDF0AB
:107DE000000EE8CFDEF081EC57F0020E0001D76FF5
:107DF000000E65EC53F0000182B007D0E90EDF6F92
:107E00006E0EE06F81EC57F006D06D0EDF6F720ED4
:107E1000E06F81EC57F0030E0001D76F000E65ECA8
:107E200053F0000182B207D0DD0EDF6F6E0EE06FFF
:107E300081EC57F006D0610EDF6F720EE06F81ECBF
:107E400057F00BEC4AF00009D8A4FBD72AEC53F00A
:107E500022D7020EBFEC55F0010E0001D76F000EC5
:107E600065EC53F00001F20EDF6F720EE06F81ECF3
:107E700057F0020E0001D76F000E65EC53F07CD86E
:107E80000009D8B473D0010EBFEC55F024EC00F01B
:107E90000001BA6FBA05D8B458D0030ED76F000EE0
:107EA00065EC53F030D00001D00EDF6F700EE06F44
:107EB00081EC57F03CD000018A0EDF6F6E0EE06F50
:107EC00081EC57F034D00001990EDF6F6E0EE06F39
:107ED00081EC57F02CD00001CD0EDF6F6E0EE06FFD
:107EE00081EC57F024D00001790EDF6F720EE06F45
:107EF00081EC57F01CD00001F50EDF6F710EE06FC2
:107F000081EC57F014D00001BA51140ACCE0010AF8
:107F1000D2E00B0AD8E0010ADEE03F0AE4E0010A01
:107F2000EAE0FD0EDF6F700EE06F81EC57F0040E9B
:107F30000001D76F000E65EC53F00001EE0EDF6F0D
:107F4000700EE06F81EC57F011D0010E0001D76F79
:107F50000B0E65EC53F00001290EDF6F700EE06F21
:107F600081EC57F0010EE8CF29FF010C040EBFECA5
:107F700055F00F01296B000C9AEC4AF0F7EC4AF02F
:107F80000009D8B4000C0001360EBB6F0F0EBC6F99
:107F900065EC4DF0006E00C002F0036A0350021061
:107FA000D8A408D00001C10EDF6F700EE06F81EC25
:107FB00057F0000C38CFE8FF3C0B3C0A0001D8B466
:107FC00007D0890EDF6F720EE06F81EC57F0000C66
:107FD000010EDF6F730EE06F81EC57F0010C0001B2
:107FE0008D0EBE6F000EBF6FC06B5BEC01F0006EBC
:107FF00000C002F0036A035002100001D8B421D07F
:10800000010E896F8A6B00018D0EBE6F000EBF6F6F
:10801000010EC06F5BEC01F0006E00C002F0036A5D
:1080200003500210D8B405D00001892B000E8A231A
:10803000EAD700018D0EBE6F000EBF6FC06B5BEF05
:1080400001F0896B8A6B120095C0E8FF500AD8A432
:108050000AD096C0E8FF520AD8A405D097C0E8FF1E
:10806000470AD8B4010C95C0E8FF440AD8A4000C14
:1080700096C0E8FF360AD8A4000C97C0E8FF340A7F
:10808000D8A4000C00019F51AB0ED8B4A019020E69
:10809000D8B4A119D8B4A251D8B4050CAB0E9F190D
:1080A000AD0ED8B4A019020ED8B4A119D8B4A251FB
:1080B000D8B4040C9F51D8B4A051030ED8B4A11960
:1080C000D8B4A251D8B4030CE00E9F19B40ED8B4A2
:1080D000A019020ED8B4A119D8B4A251D8B4020C78
:1080E000000CBA00119C11980001BE6B0FD000016A
:1080F000BC5156EC51F0006E0001BE51BA25E96E3C
:10810000000EBB21EA6E00C0EFFFBE2B11BC02D0F7
:1081100011A8EDD70001BE51BA25E96E000EBB21B2
:10812000EA6E000EEF6A1200BA00E16ABCC0D9FF25
:10813000BDC0DAFFD9CFE9FFDACFEAFFEE6AEE6A17
:10814000EE6AED6A46D00A0E046E056A066A076A90
:10815000D9CFE9FFDACFEAFFEECF00F0EECF01F0A2
:10816000EECF02F0EECF03F084EC56F000C0DEFF5D
:1081700001C0DEFF02C0DEFF03C0DDFFDD52DD52C5
:10818000E1500001BA25E96E000EBB21EA6EEF5006
:10819000006E016AD00E0026FF0E0122026A036AF9
:1081A000DE500024046EDE500120056EDE500220F9
:1081B000066EDD500320076EDD52DD5204C0DEFF87
:1081C00005C0DEFF06C0DEFF07C0DDFFDD52DD5269
:1081D000E12AE1500001BA25E96E000EBB21EA6EEA
:1081E000EF50006E300E005CD8A00CD0E150BA25E4
:1081F000E96E000EBB21EA6EEF50006E3A0E005C95
:10820000D8A0A1D7E150D8B4000C010C0001BA6F7E
:10821000030ED76F000E65EC53F09DEC53F051D078
:108220000001D40EDF6F720EE06F81EC57F09AEF11
:1082300053F00001B60EDF6F720EE06F81EC57F065
:108240009AEF53F00001520EDF6F720EE06F81EC77
:1082500057F09AEF53F00001980EDF6F720EE06F47
:1082600081EC57F09AEF53F00001430EDF6F720E6E
:10827000E06F81EC57F09AEF53F00001A70EDF6F2B
:10828000720EE06F81EC57F09AEF53F00001340E5C
:10829000DF6F720EE06F81EC57F09AEF53F0000140
:1082A000E30EDF6F720EE06F81EC57F09AEF53F040
:1082B0000001C50EDF6F720EE06F81EC57F09AEF90
:1082C00053F00001BA51010AABE0030AB2E0010A1F
:1082D000B9E0070AC0E0010AC7E0030ACEE0010ADC
:1082E000D5E00F0ADCE0010AE3E01D0EDF6F730E3C
:1082F000E06F81EC57F09AEF53F0BA000001BC0533
:10830000D8B498EC53F00001D76B000E65EC53F035
:108310000001F50EDF6F6E0EE06F89C0BFF08AC0FE
:10832000C0F0BAC0BDF0BBC0BEF0BD0EE8CFDDF0FE
:10833000000EE8CFDEF081EC57F0010E0001D76FA0
:10834000000E65EC53F000011D0EDF6F730EE06F41
:1083500081EC57F0010E0001D76F000E65EC53F071
:108360000001BB51BA11D8A408D07B0EDF6F6E0E8E
:10837000E06F81EC57F09AEF53F08DC0E8FF09EC05
:1083800056F08EC0E8FF200AD8A41ED08FC0E8FFA8
:10839000200AD8A419D090C0E8FF200AD8A414D08D
:1083A00091C0E8FF200AD8A40FD092C0E8FF200AAD
:1083B000D8A40AD093C0E8FF200AD8A405D094C05E
:1083C000E8FF200AD8B404D08EC0E8FF09EC56F0CC
:1083D0008FC0E8FF200AD8A419D090C0E8FF200A77
:1083E000D8A414D091C0E8FF200AD8A40FD092C01E
:1083F000E8FF200AD8A40AD093C0E8FF200AD8A436
:1084000005D094C0E8FF200AD8B404D08FC0E8FF9C
:1084100009EC56F090C0E8FF200AD8A414D091C00F
:10842000E8FF200AD8A40FD092C0E8FF200AD8A401
:108430000AD093C0E8FF200AD8A405D094C0E8FF72
:10844000200AD8B404D090C0E8FF09EC56F091C0DF
:10845000E8FF200AD8A40FD092C0E8FF200AD8A4D1
:108460000AD093C0E8FF200AD8A405D094C0E8FF42
:10847000200AD8B404D091C0E8FF09EC56F092C0AD
:10848000E8FF200AD8A40AD093C0E8FF200AD8A4A5
:1084900005D094C0E8FF200AD8B404D092C0E8FF09
:1084A00009EC56F093C0E8FF200AD8A405D094C088
:1084B000E8FF200AD8B404D093C0E8FF09EC56F0D6
:1084C00094C0E8FF200AD8B404D094C0E8FF09ECB7
:1084D00056F02E0E09EC56F095C0E8FF09EC56F068
:1084E00096C0E8FF09EC56F097C0E8FF09EC56F09B
:1084F0009AEF53F0C9000001CE6F040ED76F000E43
:1085000065EC53F00001CC51D76FCA5144EC54F0E4
:10851000050E0001D76F000E65EC53F00001060E4A
:10852000DF6F6F0EE06FC9C000F0016A00C0D5F0C8
:1085300001C0D6F0CEC000F0016A00C0D3F001C087
:10854000D4F033CFD1F0D26B0D0ECF6FD06BCF0EF6
:10855000E8CFDDF0000EE8CFDEF081EF57F00BEC56
:108560004AF012A031D000018B518C11D8B41AD02E
:108570008B51010A8C11D8B412D000018D0EBE6F40
:10858000000EBF6F020EC06F5BEC01F0006E00C00A
:1085900002F0036A03500210D8B404D000018B0724
:1085A000000E8C5B020EE8CF29FF8BC0BAF08CC0A6
:1085B000BBF0010E0001BC6FA1DE00015E0EC06FBA
:1085C000010EC16FA5EC55F011AE3BD089C002F091
:1085D0008AC003F08BC000F08CC001F00350015C36
:1085E00002E10250005CD8B01AD000018B518C110E
:1085F000D8B412D000018D0EBE6F000EBF6F010EF9
:10860000C06F5BEC01F0006E00C002F0036A035023
:108610000210D8B404D000018B2B000E8C23020E64
:10862000E8CF29FF8BC0BAF08CC0BBF0010E00016F
:10863000BC6F64DE00015E0EC06F010EC16FA5EC61
:1086400055F012A2120000DD006E020E005CD8A0F0
:108650001CD000018D0EBA6F000EBB6F58EC03F0FA
:10866000010EE8CF29FF8BC0BAF08CC0BBF000012F
:10867000BC6B44DE00018B518C11D8A4B1EF48F0E3
:10868000030E0001C96FB3EF48F0010E0001D76F70
:10869000000E65EC53F098EC53F00001DF0EDF6F35
:1086A000700EE06F81EC57F09AEC53F00001DC0E95
:1086B000C06F050EC16FA5EC55F08BC0BAF08CC031
:1086C000BBF0010E0001BC6F19D6010E0001C96F8D
:1086D000000EC4EC48F0119893EC52F0010EC7EC78
:1086E00051F0040EC7EC51F0010EC7EC51F0010E31
:1086F000C7EC51F0000EC7EC51F0000EC7EC51F082
:10870000200EC7EC51F0120EC7EC51F0220EC7EC50
:1087100051F00001230EC96F720ECA6F46EC52F081
:10872000220EC7EC51F0000EC7EC51F0010EC7EC61
:1087300051F0010EC7EC51F0000EC7EC51F0000EE5
:10874000C7EC51F0200EC7EC51F0220EC7EC51F0EF
:108750000001BC0EC96F6E0ECA6F46EC52F0220EBD
:10876000C7EC51F0000EC7EC51F0010EC7EC51F010
:10877000010EC7EC51F0000EC7EC51F0000EC7EC33
:1087800051F0200EC7EC51F0220EC7EC51F0000161
:10879000480EC96F6E0ECA6F46EC52F0220EC7EC3F
:1087A00051F0000EC7EC51F0010EC7EC51F0010E74
:1087B000C7EC51F0000EC7EC51F0000EC7EC51F0C1
:1087C000200EC7EC51F0220EC7EC51F00001260E2E
:1087D000C96F6E0ECA6F46EC52F0220EC7EC51F014
:1087E000000EC7EC51F0010EC7EC51F0010EC7ECC2
:1087F00051F0000EC7EC51F0000EC7EC51F0200E06
:10880000C7EC51F0220EC7EC51F000016A0EC96F9F
:108810006E0ECA6F46EC52F0220EC7EC51F0000EFD
:10882000C7EC51F0010EC7EC51F0010EC7EC51F04E
:10883000000EC7EC51F0000EC7EC51F0200EC7EC53
:1088400051F0220EC7EC51F00001590EC96F6E0EA7
:10885000CA6F46EC52F0220EC7EC51F0000EC7EC86
:1088600051F0010EC7EC51F0010EC7EC51F0000EB3
:10887000C7EC51F0000EC7EC51F0200EC7EC51F0E0
:10888000220EC7EC51F00001370EC96F6E0ECA6F91
:1088900046EC52F0220EC7EC51F0000EC7EC51F03E
:1088A000010EC7EC51F0010EC7EC51F0000EC7EC01
:1088B00051F0000EC7EC51F0200EC7EC51F0220E23
:1088C000C7EC51F00001AB0EC96F6E0ECA6F46ECDB
:1088D00052F0220EC7EC51F0000EC7EC51F000012F
:1088E000BA6B8D0EBE6F000EBF6FC06B5BEC01F0FC
:1088F000006E00C002F0036A03500210D8B481D0A9
:108900000001BA2B24EC40F00009D8B469D0010E64
:10891000C7EC51F0010EC7EC51F00001BA51C7ECA1
:1089200051F0026A010E036EBAC000F0016A2AEC2F
:1089300057F00450C7EC51F00A0E0001BA6103D0A1
:10894000200EC7EC51F0220EC7EC51F08DC0E8FFAD
:10895000C7EC51F08EC0E8FFC7EC51F08FC0E8FFC4
:10896000C7EC51F090C0E8FFC7EC51F091C0E8FFB0
:10897000C7EC51F092C0E8FFC7EC51F093C0E8FF9C
:10898000C7EC51F094C0E8FFC7EC51F02E0EC7ECD5
:1089900051F095C0E8FFC7EC51F096C0E8FFC7EC76
:1089A00051F097C0E8FFC7EC51F0220EC7EC51F030
:1089B000000EC7EC51F00001C96BBA5189C000F03C
:1089C0008AC001F0005CCA6F0150D8A00104CB6FCF
:1089D00000EECCF089C0EEFF8AC0EDFF000E8BDD0B
:1089E00000018D0EBE6F000EBF6F010EC06F5BECFD
:1089F00001F0006E00C002F0036A03500210D8A418
:108A00007FD700018D0EBE6F000EBF6FC06B5BEC99
:108A100001F0000EC7EC51F01188000EC7EC51F0C8
:108A2000A4EC52F02DD6BA00010E0001C96F000E61
:108A3000ABDB119893EC52F0010EC7EC51F0040E31
:108A4000C7EC51F000018D0EC96F000ECA6F120EF7
:108A5000CB6FCC6B900ECD6F190ECE6FCF6B7BECC6
:108A600007F0010E0001C76FC86BC96B010ECA6F1A
:108A7000CB6BCC6BCD6B120E3EDD010EC7EC51F013
:108A8000010EC7EC51F00001BA51C7EC51F00001E2
:108A9000BB51C7EC51F0120EC7EC51F0220EC7ECDF
:108AA00051F00001C16B0001C1510AEE23F0E9262B
:108AB000000EEA22EF50C7EC51F00001C12B0F0E5F
:108AC000C165F1D7220EC7EC51F0200EC7EC51F072
:108AD00035CAE8FFC7EC51F036CAE8FFC7EC51F0E1
:108AE000200EC7EC51F038CAE8FFC7EC51F039CA84
:108AF000E8FFC7EC51F0000EC7EC51F00001BE6B6F
:108B00000001BE5104EC06F00009D8B45BD10001AD
:108B1000C74BC82B2BCFC9F0C7C0CAF0C8C0CBF019
:108B2000CC6BCD6B2CCFE8FFE6DC010E0001BE6FF5
:108B3000BF6B43D10001BF39E846E00B020FC26FA3
:108B4000C2510AEE23F0E926000EEA22EF50D8B413
:108B500032D1010EC7EC51F0010EC7EC51F000010B
:108B6000C2510AEE3FF0E926000EEA22EF50C7ECB0
:108B700051F00001C2510AEE40F0E926000EEA224F
:108B8000EF50C7EC51F00001C2510AEE3FF0E92668
:108B9000000EEA22EF50006EC2510AEE40F0E926C4
:108BA000000EEA22EF50C66F00C0C5F0000EC65D91
:108BB0000A0ED8B4C55DD8B003D0200EC7EC51F072
:108BC0000001000EC65D640ED8B4C55DD8B003D0F8
:108BD000200EC7EC51F00001030EC65DE80ED8B4BC
:108BE000C55DD8B003D0200EC7EC51F0220EC7EC03
:108BF00051F00001C06B030EC16F0001C251C1C032
:108C000000F0016A0026000E0122230E0024E96E06
:108C10000A0E0120EA6EEF50A00AD8B411D0C2515A
:108C2000C1C000F0016A0026000E0122230E0024BC
:108C3000E96E0A0E0120EA6EEF50200AD8A408D08F
:108C40000001C02B1AD0200EC7EC51F00001C00764
:108C50000001C051D8A4F7D70001C251C1C000F033
:108C6000016A0026000E0122230E0024E96E0A0E7E
:108C70000120EA6EEF50C7EC51F00001C12B120E3B
:108C8000C165BBD7220EC7EC51F00001C051D8B46A
:108C900006D0200EC7EC51F00001C007F6D7000146
:108CA000C2510AEE23F0E926000EEA22EF50006ED0
:108CB000800E005CD8A004D0200EC7EC51F036D056
:108CC0002A0EC7EC51F032D0440EC7EC51F0450EDD
:108CD000C7EC51F04C0EC7EC51F04DD0530EC7EC21
:108CE00051F0450EC7EC51F0510EC7EC51F043D096
:108CF000500EC7EC51F0520EC7EC51F0470EC7ECC6
:108D000051F039D0550EC7EC51F0530EC7EC51F06D
:108D1000520EC7EC51F02FD0520EC7EC51F0450E59
:108D2000C7EC51F04C0EC7EC51F025D00001C251F8
:108D30000AEE23F0E926000EEA22EF50006E070E3D
:108D4000001600C002F0036A0BD00250BDE0010A19
:108D5000C5E0030ACDE0010AD5E0070ADDE002D054
:108D60000350F3E0550EC7EC51F04E0EC7EC51F036
:108D70004B0EC7EC51F00001C2510AEE23F0E92678
:108D8000000EEA22EF50006EC00E005CD8A004D0A6
:108D90003C0EC7EC51F003D0200EC7EC51F0200E72
:108DA000C7EC51F0200EC7EC51F0200EC7EC51F08B
:108DB000000EC7EC51F00001BF2B070E0001BF658C
:108DC000B9D69ED6010EC7EC51F0010EC7EC51F09A
:108DD00032EC06F000C0C3F001C0C4F00001C35182
:108DE000C7EC51F00001C451C7EC51F00001100E66
:108DF000C96F730ECA6F46EC52F0000EC7EC51F00B
:108E0000000EC7EC51F01188000EC7EC51F0A4EC35
:108E100052F0A7D1BCC0BEF0BDC0BFF00001C06B16
:108E20005BEC01F0006E00C002F0036A0350021018
:108E3000D8B4000CD968D92ABCC0E1FFBDC0E2FF9C
:108E4000D950080AD8A41ED000EE08F0E150E92657
:108E5000E250EA22EF50500AD8A414D000EE09F0F4
:108E6000E150E926E250EA22EF50520AD8A40AD093
:108E700000EE0AF0E150E926E250EA22EF50470AFC
:108E8000D8B4010C0001BA51D924E96E000ED9BE44
:108E9000FF0EBB21EA6EEF50D8B436D00001BA51B4
:108EA000D924E96E000ED9BEFF0EBB21EA6EEF5049
:108EB0003F0AD8A408D0D950E124E96E000EE22080
:108EC000EA6E3F0EEF6E0001BA51D924E96E000E32
:108ED000D9BEFF0EBB21EA6EEF502A0AD8B4010CAE
:108EE000BA51D924E96E000ED9BEFF0EBB21EA6E3D
:108EF000EF50006ED950E124E96E000EE220EA6ED8
:108F0000EF500018D8B497D7BCC0BEF0BDC0BFF0BA
:108F1000010E0001C06F5BEC01F084D7010E00016F
:108F2000C96F000E31D9119893EC52F0BAC0E1FF2D
:108F3000BBC0E2FF00EE12F0E150E926E250EA2267
:108F4000EECFC3F0EECFC4F0EECFC5F0EECFC6F05B
:108F50000001BF6BC06BBC6BFE0E046E056A066A37
:108F6000076AC3C000F0C4C001F0C5C002F0C6C0AB
:108F700003F029EC56F000C0C1F001C0C2F0C1C03E
:108F8000BDF0C2C0BEF0FE0E046E056A066A076A36
:108F9000C3C000F0C4C001F0C5C002F0C6C003F0F9
:108FA00029EC56F00750041005100610D8B402D072
:108FB000C14BC22B0001C107D8A0C207E1CFC7F047
:108FC000E2CFC8F0A5EC05F00001C651C311C411F1
:108FD000C511D8B444D00001C305C411C511C611D0
:108FE000D8B411880AEE23F0BF51E926C051EA2215
:108FF000EF50C7EC51F00001C307000EC45BC55B26
:10900000C65BBC2BBF4BC02BC051020ABF11D8A4FA
:109010000FD0BAC0C7F0BBC0C8F097EC03F0BAC01D
:10902000C7F0BBC0C8F0A5EC05F00001BF6BC06B7A
:109030000001BC51FE0AD8A4C7D7C107D8A0C207F7
:10904000C96BC1C0CAF0C2C0CBF0BDC0CCF0BEC0BD
:10905000CDF0000E7BEC42F00001BC6BB5D7A4EC68
:1090600052F040EF43F0BA000001BD6FBBC0C3F047
:10907000BCC0C4F0010EC96F000E86D8119893ECE5
:1090800052F00001BA51C96FC3C0CAF0C4C0CBF0DE
:10909000BBC0CCF0BCC0CDF0BD517BEC42F00001B8
:1090A000BD51C16FC26BBA51BF6FC06B8D0EC96F1E
:1090B000000ECA6FBD51CB6FBA51CC6FCD6BCE6B6A
:1090C000010ECF6F7BEC07F023CABDF024CABAF0C3
:1090D0000001C307D8A0C407BD51D8B412D0020EF6
:1090E000BE6F0001BE510AEE23F0E926000EEA220F
:1090F000EF50C7EC51F00001BE2BBE51D8B4C1D720
:10910000F0D70001BF51C96FC3C0CAF0C4C0CBF0D3
:10911000BBC0CCF0BCC0CDF0C1517BEC42F0020E24
:109120000001BE6F0001BA51BE5DD8B00DD0000184
:10913000BE510AEE23F0E926000EEA22EF50C7ECFA
:1091400051F00001BE2BEED711880001BA510AEE92
:1091500023F0E926000EEA22EF50C7EC51F0A4EC10
:1091600052F00001C96B000E0FD0BA00BBC0F3FF74
:10917000BCC0F4FF010E0001C96F000E05D80A0E35
:10918000BFEC55F0EED7C900D96ED950D8B421D074
:1091900034CFE8FF490AD8A4D9CF34FF1AD0D59EDE
:1091A00080921200D59E80821200020EE8CF28FF26
:1091B000119AD768D668D58E1200030EE8CF28FF23
:1091C0001196119AD768D668D58E1200D59E8092D6
:1091D00012000001C951E3E0010AE4E0030AE5E0FE
:1091E000010AEBE0F3D71198808293EC52F034CF70
:1091F000E8FF7BEC52F02C0EC7EC51F0D7D0000109
:10920000290EC96F700ECA6F46EC52F0E3D0000110
:109210008A0EC96F700ECA6F46EC52F0DBD00001A7
:109220009A0EC96F700ECA6F46EC52F0D3D000018F
:10923000CC0EC96F6F0ECA6F46EC52F0CBD0000156
:10924000C00EC96F6F0ECA6F46EC52F0C3D000015A
:10925000E50EC96F6F0ECA6F46EC52F0BBD000012D
:10926000480EC96F700ECA6F46EC52F0B3D00001C1
:10927000B30EC96F6F0ECA6F46EC52F0ABD000014F
:10928000550EC96F6F0ECA6F46EC52F0A3D00001A5
:10929000680EC96F700ECA6F46EC52F09BD0000189
:1092A000590EC96F700ECA6F46EC52F093D0000190
:1092B000040EC96F700ECA6F46EC52F08BD00001DD
:1092C000F60EC96F6F0ECA6F46EC52F083D00001E4
:1092D0007B0EC96F700ECA6F46EC52F07BD0000156
:1092E000680EC96F6F0ECA6F46EC52F073D0000162
:1092F000350EC96F700ECA6F46EC52F06BD000018C
:109300002C0EC96F700ECA6F46EC52F063D000018C
:109310008A0EC96F6F0ECA6F46EC52F05BD0000127
:10932000740EC96F6F0ECA6F46EC52F053D0000135
:109330001E0EC96F700ECA6F46EC52F04BD0000182
:10934000A30EC96F6F0ECA6F46EC52F043D00001F6
:10935000140EC96F700ECA6F46EC52F03BD000017C
:109360004A0EC96F6F0ECA6F46EC52F0060E7BECC8
:1093700052F02E0EC7EC51F0080E7BEC52F02E0E80
:10938000C7EC51F0190E7BEC52F024D000012E0EE8
:10939000C96F6F0ECA6F46EC52F01CD00001D70E99
:1093A000C96F6F0ECA6F46EC52F014D034CFE8FF8D
:1093B000000FF4E6B50FF2E74B0F020D900EF32409
:1093C000F66E6D0EF420F76E0900F5500900F5CF2A
:1093D000FAFFF96E320E0001C06FC16BA5EC55F0BB
:1093E0002C0EC7EC51F02CCFE8FF7BEC52F02C0E8A
:1093F000C7EC51F02BCFE8FF7BEC52F011880D0E3B
:10940000C7EC51F0A4EC52F080920F01346B1200C3
:1094100082A0080C090C046A056A066A076AC282FF
:10942000C2B2FED7C450016E006AC3500024026E5F
:10943000000E0120036E000102C0C1F003C0C2F0A3
:10944000000EC2BFFF0EC36FC46F071808E10650BD
:10945000C31905E10550C21902E10450C119D8B47D
:109460000CD0C1C004F0C2C005F0C3C006F0C4C037
:1094700007F0C282C2A2D6D7FDD70001C06B1290FE
:109480001292119E9A0EC125C56FFC0EC221C66FA5
:109490005EEC57F00150800A800F100ED8B4005CCB
:1094A000D8B002D0128025D000012F0EC125C56F83
:1094B000FD0EC221C66F5EEC57F00150800A800F8E
:1094C000100ED8B4005CD8B002D0128212D00001C5
:1094D000C10EC125C56FFD0EC221C66F5EEC57F0EF
:1094E0000150800A800F100ED8B4005CD8B004D0B0
:1094F000118E010E0001C06F0001C0511200000169
:10950000756B766BFF0E24EC56F0FE0AD8B4010C96
:10951000000175C000F076C001F00028756F02E10F
:109520000128766F030E015CE80ED8B4005CD8B059
:10953000000CE8D788D882840001BB6BBC6BFF0E9F
:1095400024EC56F00001BB4BBC2B000EBC5D0A0E98
:10955000D8B4BB5DD8A0F3D78294F36AF46AF34A17
:10956000F42AC30EF45C500ED8B4F35CD8A0F7D73D
:1095700074D80009D8B4000C0001F66BF76BF86BD7
:10958000F96B770EF2DB19CAE8FF050AD8A405D0FB
:109590007CD80009D8B4000C24D00001756B766B20
:1095A000010EE8CF19FA0A011953D8B41AD00001F4
:1095B000F66BF76BF86BF96B690ED7DB0001F66B96
:1095C000F76BF86BF96B770ED0DB00017651270A49
:1095D000100ED8B47519D8B4000C752B000E762374
:1095E000E2D770D80009D8B4000C32D8010C2BD8BF
:1095F00082840001BB6BBC6BFF0E24EC56F00001B3
:10960000BB4BBC2B000EBC5D0A0ED8B4BB5DD8A012
:10961000F3D78294F36AF46AF34AF42AC30EF45C33
:10962000500ED8B4F35CD8A0F7D717D80009D8B437
:10963000000C2BD80009D8B4000C44D80009D8B4C9
:10964000000C06D8010CC696C694C682C6901200BD
:10965000C696C694C692C6801200640E0001BD6F05
:109660000001BD07BD29D8B4010CF66BF76BF86B90
:10967000F96B400E7ADB19CA00F00004D8B4010C73
:109680000001BD51D8B4000CEBD70001756B766BAF
:10969000010EE8CF19FA0A011953D8B4010C0001E0
:1096A000F66BF76BF86BF96B410E5FDB00017651DF
:1096B000270A100ED8B47519D8B4000C752B000EFB
:1096C0007623E9D7640E0001BD6F0001BD07BD29F7
:1096D000D8B4010CF66BF76BF86B020EF96F500EF5
:1096E00044DB0A011953D8B4010C0001BD51D8B4B0
:1096F000000CEBD70001F66BF76BF86BF96B4A0EB9
:1097000034DBFDDE0009D8B4000C11900001080E16
:10971000DF6F120EE06F81EC57F00001340EDF6F47
:10972000110EE06FFF0E24EC56F0006E00C002F048
:10973000036A02C0A5F003C0A6F0A50EE8CFDDF0D5
:10974000000EE8CFDEF081EC57F00001180EDF6F5D
:10975000110EE06FFF0E24EC56F0006E00C002F018
:10976000036A02C0A5F003C0A6F0A50EE8CFDDF0A5
:10977000000EE8CFDEF081EC57F00001FC0EDF6F49
:10978000100EE06FFF0E24EC56F0006E00C002F0E9
:10979000036A02C0A5F003C0A6F0A50EE8CFDDF075
:1097A000000EE8CFDEF081EC57F000018C0EDF6F89
:1097B000100EE06FFF0E24EC56F0006E00C002F0B9
:1097C000036A02C0A5F003C0A6F0A50EE8CFDDF045
:1097D000000EE8CFDEF081EC57F00001700EDF6F75
:1097E000100EE06FFF0E24EC56F0006E00C002F089
:1097F000036A02C0A5F003C0A6F0A50EE8CFDDF015
:10980000000EE8CFDEF081EC57F00001540EDF6F60
:10981000100EE06FFF0E24EC56F0006E00C002F058
:10982000036A02C0A5F003C0A6F0A50EE8CFDDF0E4
:10983000000EE8CFDEF081EC57F00001380EDF6F4C
:10984000100EE06FFF0E24EC56F0006E00C002F028
:10985000036A02C0A5F003C0A6F0A50EE8CFDDF0B4
:10986000000EE8CFDEF081EC57F000011C0EDF6F38
:10987000100EE06FFF0E24EC56F0006E00C002F0F8
:10988000036A02C0A5F003C0A6F0A50EE8CFDDF084
:10989000000EE8CFDEF081EC57F00001000EDF6F24
:1098A000100EE06FFF0E24EC56F0006E00C002F0C8
:1098B000036A02C0A5F003C0A6F0A50EE8CFDDF054
:1098C000000EE8CFDEF081EC57F00001A80EDF6F4C
:1098D000100EE06FFF0E24EC56F0006E00C002F098
:1098E000036A02C0A5F003C0A6F0A50EE8CFDDF024
:1098F000000EE8CFDEF081EC57F00001E00EDF6FE4
:10990000100EE06FFF0E24EC56F0006E00C002F067
:10991000036A02C0A5F003C0A6F0A50EE8CFDDF0F3
:10992000000EE8CFDEF081EC57F00001A40EDF6FEF
:10993000110EE06FFF0E24EC56F0006E00C002F036
:10994000036A02C0A5F003C0A6F0A50EE8CFDDF0C3
:10995000000EE8CFDEF081EC57F00001880EDF6FDB
:10996000110EE06FFF0E24EC56F0006E00C002F006
:10997000036A02C0A5F003C0A6F0A50EE8CFDDF093
:10998000000EE8CFDEF081EC57F000016C0EDF6FC7
:10999000110EE06FFF0E24EC56F0006E00C002F0D6
:1099A000036A02C0A5F003C0A6F0A50EE8CFDDF063
:1099B000000EE8CFDEF081EC57F00001C40EDF6F3F
:1099C000100EE06FFF0E24EC56F0006E00C002F0A7
:1099D000036A02C0A5F003C0A6F0A50EE8CFDDF033
:1099E000000EE8CFDEF081EC57F00001500EDF6F83
:1099F000110EE06FFF0E24EC56F0006E00C002F076
:109A0000036A02C0A5F003C0A6F0A50EE8CFDDF002
:109A1000000EE8CFDEF081EC57F01180010C000160
:109A2000F66BF76BF86BF96B490E9FD968DD00098F
:109A3000D8B4000C11900001D30EDF6F110EE06F4F
:109A400081EC57F00001A56BA66B0001C00EDF6F23
:109A5000110EE06FFF0E24EC56F0006E00C002F015
:109A6000036A02C0A9F003C0AAF0A5C0A7F0A6C06F
:109A7000A8F0A70EE8CFDDF0000EE8CFDEF081EC15
:109A800057F00001A54BA62B000EA65D110ED8B411
:109A9000A55DD8A0DAD71180010CA5000001A56B47
:109AA000A66BA76BA86B4D0E72D9A5C0E1FFA6C02F
:109AB000E2FF00EE01F0E150E926E250EA2219CA85
:109AC000EFFF1ACAE7FF010CBB000001756B766B54
:109AD000010EE8CF19FA0A011953D8B410D00001C9
:109AE000BD6BBE6BBF6BC06B7A0E68D90001751D74
:109AF0007611D8B4000C752B000E7623ECD7BBC0C2
:109B0000E1FFBCC0E2FF00EE03F0E150E926E250C5
:109B1000EA221ACAEFFF00EE02F0E150E926E25015
:109B2000EA221BCAEFFF00EE01F0E150E926E25005
:109B3000EA221CCAEFFF1DCAE7FF010CEC0000017E
:109B4000090ED890EC37ED37EE37EF37E82EF9D71E
:109B5000EEC0F6FFEFC0F7FFECC0F3FFEDC0F4FF7F
:109B6000F6CFF6F0F7CFF7F0F3CFF8F0F4CFF9F047
:109B7000510EFBD8C4DC0009D8B4000CF2C0E1FFE0
:109B8000F3C0E2FF006A016A026A036AC968C7A0FB
:109B9000FED70001F151F011D8A403D0C9CFE6FFE0
:109BA00006D0C9CFE7FF0001F007D8A0F107002ACF
:109BB000000E012202220322035C08E1000E025C77
:109BC00005E1020E015C02E1000E005CD8A0DED7C8
:109BD000FF0E24EC56F0FF0E24EC56F0010CCF00E3
:109BE0000001090ED890CF37D037D137D237E82EC1
:109BF000F9D7D1C0F3FFD2C0F4FFCFC0F6FFD0C079
:109C0000F7FFF3CFF6F0F4CFF7F0F6CFF8F0F7CF99
:109C1000F9F0510EAAD873DC0009D8B4150CD3C0E2
:109C2000E1FFD4C0E2FFD96AC968C7A0FED7C9CF97
:109C3000E6FFD92EF9D7C968C7A0FED7C9CFE6FF7E
:109C4000D92EF9D7FF0E24EC56F0FF0E24EC56F077
:109C5000010CA5000001090ED890A537A637A7373B
:109C6000A837E82EF9D7A7C0F6FFA8C0F7FFA5C010
:109C7000F3FFA6C0F4FFF6CFF6F0F7CFF7F0F3CF7F
:109C8000F8F0F4CFF9F0580E70D80A011953D8A49F
:109C9000000CFF0E24EC56F0FF0E24EC56F0FE0EE6
:109CA00024EC56F00001A66BA76B0001A651A92574
:109CB000E96EA751AA21EA6EEF5024EC56F000019C
:109CC000A64BA72B020EA75D000ED8B4A65DD8A0A8
:109CD000ECD7FF0E24EC56F0FF0E24EC56F0FF0EEE
:109CE00024EC56F00001A56FFF0E24EC56F0006E38
:109CF0000028D8B4010CF8D7FB000001FF6F0A015F
:109D0000186BFF0E24EC56F00001FF5124EC56F0C6
:109D10000001FF5178D80001FC5124EC56F00001FD
:109D2000FC5171D80001FB5124EC56F00001FB51AD
:109D30006AD80001FE5124EC56F00001FE5163D8B0
:109D40000001FD5124EC56F00001FD515CD80AEEF3
:109D500018F0D890EF360A01182B18CAE8FF24EC47
:109D600056F0FF0E24EF56F0F6000001FA6FF6C031
:109D7000FBF0F7C0FCF0F8C0FDF0F9C0FEF0BDDF6D
:109D8000FF0E24EC56F0E8CF19FA1200A5000001EE
:109D9000A56FA5C0FBF0A6C0FCF0A7C0FDF0A8C051
:109DA000FEF0ABDFFF0E24EC56F0E8CF19FAFF0E01
:109DB00024EC56F0E8CF1AFA1200BD000001C16F82
:109DC000BDC0FBF0BEC0FCF0BFC0FDF0C0C0FEF0E7
:109DD00094DFFF0E24EC56F0E8CF19FAFF0E24ECC6
:109DE00056F0E8CF1AFAFF0E24EC56F0E8CF1BFA33
:109DF000FF0E24EC56F0E8CF1CFAFF0E24EC56F0D0
:109E0000E8CF1DFA1200D96E080EE16E0AEE18F0C6
:109E1000D890EF360A01D9AE02D0090E181B18AF40
:109E200003D00A01090E181BD890D936E12EEED7BF
:109E30001200EC00ECC0F6FFEDC0F7FF0F0EF76468
:109E400003D00800F55005D0F6CFE9FFF7CFEAFFC1
:109E5000EF501200DD000001E86BE96BDDC0E1FFAF
:109E6000DEC0E2FF0001E151EC6FE251ED6FE14B2A
:109E7000E22BE0DF0001E76FE751D8B4E1D1000148
:109E8000E751250AD8B404D0E751E36FE7D9EAD700
:109E90000001E469E66BE56B93D10001E051DF114D
:109EA000D8B406D0DFC0E9FFE0C0EAFF000EEF6AD9
:109EB000E8C000F0E9C001F01200E1CFE9FFE2CF15
:109EC000EAFF020EE126000EE222EF500001B1D1BE
:109ED0000001E58D75D10001E52B0A0E04D0100EAE
:109EE00001D0080E0001E46FE6CFF6FFE6CFF7FFE2
:109EF0000001E5A10DD0F7AE06D0F66CF71ED8B084
:109F0000F72AE60707D00001E591E5AD03D0F9D7C0
:109F10000001E591E4C002F0036AF6CF00F0F7CF4C
:109F200001F0C7EC56F000500001E76FE4C002F00A
:109F3000036AF6CF00F0F7CF01F0C7EC56F004C08B
:109F4000F6FF05C0F7FF010EEA6FEB6B0001EB5166
:109F5000F75C02E1EA51F65CD8A010D0E4C002F050
:109F6000036AEAC000F0EBC001F04FEC57F004C008
:109F7000EAF005C0EBF00001E607E8D70001E5A92B
:109F800005D00BD0200E0001E36F68D90001E60771
:109F9000E651800A7F0FD8B0F5D70001E5A104D0C3
:109FA0002D0EE36F5BD906D00001E5AD03D02B0E7B
:109FB000E36F54D90001E5B905D02ED0300E000171
:109FC000E36F4CD90001E607E651800A7F0FD8A065
:109FD00023D0F4D7EAC002F0EBC003F0F6CF00F0D4
:109FE000F7CF01F0C7EC56F004C000F005C001F057
:109FF000E4C002F0036AC7EC56F000500001E66FBF
:10A00000E651800A760FD8A002D0070EE62700019D
:10A01000E651300FE36F22D9E4C002F0036AEA0E82
:10A02000E96E000EEA6EEE50006EEF50016EC7EC66
:10A0300056F00550ED6E0450EF6EEE50ED10D8A4C2
:10A04000C9D7090E0001E76502D0070EE727000116
:10A05000E751300FE36F02D905D70001E651800ABE
:10A060007E0FD8A006D0200E0001E36FF7D8E607D8
:10A07000F4D7E1CFE9FFE2CFEAFF020EE126000EBE
:10A08000E222EF500001E76FE751E36FE7D8EAD62D
:10A09000E1CFE9FFE2CFEAFF020EE126000EE22265
:10A0A000EECF00F0EDCF01F000C077F001C078F006
:10A0B0000001E76B77C000F078C001F00001E751C4
:10A0C0000024026E000E0120036E02C0F6FF03C0E2
:10A0D000F7FF0F0EF76403D00800F55005D0F6CF58
:10A0E000E9FFF7CFEAFFEF500009D8B403D0000131
:10A0F000E72BE0D70001E451E76102D0E751E46FBC
:10A100000001E451E6BF1ED0FF0AE625D8A01AD010
:10A11000200E0001E36FA2D8E607F2D7000177C056
:10A1200000F078C001F00028776F02E10128786F15
:10A1300000C0ECF001C0EDF07DDE0001E76FE751FB
:10A14000E36F8CD80001E407E429D8B48BD6E6D7B6
:10A15000E1C0ECF0E2C0EDF06DDE2A0AD8A40ED02A
:10A16000E1CFE9FFE2CFEAFF020EE126000EE22294
:10A17000EF500001E46FE14BE22B22D00001E151EE
:10A18000EC6FE251ED6FE14BE22B54DED00F00019A
:10A19000E46FE1C0ECF0E2C0EDF04CDE0001E76FEF
:10A1A0002F0EE7650DD03A0EE7610AD0E4510A0D93
:10A1B000E751F324D00FDED70001E5B52DD0E589B6
:10A1C0000001E151EC6FE251ED6FE14BE22B32DE29
:10A1D0000001E76FE75101E160D62A0A01E16DD67F
:10A1E000010A01E175D6050AB3E01E0AE5E0680A36
:10A1F00001E175D63B0A01E130D7070A01E16BD6D0
:10A200000B0A01E16ED61C0A01E142D7060A01E100
:10A210006BD60D0A01E163D62F0E0001E7650BD066
:10A220003A0EE76108D0E585E6510A0DE751F324BF
:10A23000D00FE66FC5D70001E751E36F0FD812D6F4
:10A240000001E051DF11D8B406D0DFC0E9FFE0C063
:10A25000EAFF000EEF6A0001E72B13D0E84BE92B71
:10A26000E051DF11D8B409D0DFC0E9FFE0C0EAFF58
:10A27000E3C0EFFFDF4BE02B12000001E35109EFD9
:10A2800056F0E8C000F0E9C001F012000001AB6F29
:10A29000B6D9BCD9C1D91198119CABC027FF120007
:10A2A000AED9B4D9B9D981B01200FDD70001BF6FC2
:10A2B0001198119CC16B080EC06F80A4FED7ACD959
:10A2C0000001880EC26F130EC36F000EC46FC56FFE
:10A2D000000180A44BD0C207000EC35BC45BC55B0A
:10A2E000C551C211C311C411D8A4F2D7118897D98E
:10A2F000460E0001CE6FCF6B66EC55F08DD9E8D7D6
:10A300000001D890C133C007880E006E130E016E95
:10A31000000E026E036E80A4FED70006000E015AE6
:10A32000025A035A0350001001100210D8A402D0A0
:10A33000118C000C80A603D0800E0001C127880E6E
:10A34000006E130E016E000E026E036E80B4FED717
:10A350000006000E015A025A035A03500010011061
:10A360000210D8A402D0118C000C0001C051D8A456
:10A37000C7D70001BF51D8A406D0E20ECE6F040E9D
:10A38000CF6F66EC55F04BD90001C15112000001AE
:10A39000CC6F080ECD6F119C39D980A6FED711A8BD
:10A3A00032D0C80E0001CE6FCF6B66EC55F0880E30
:10A3B000006E130E016E000E026E036E80B6FED7A5
:10A3C0000006000E015A025A035A035000100110F1
:10A3D0000210D8A402D0118C000C880E006E130E4F
:10A3E000016E000E026E036E80A6FED70006000E00
:10A3F000015A025A035A0350001001100210D8A447
:10A4000002D0118C000C05D9500E0001CE6FCF6B1D
:10A4100066EC55F00001CD51D8B418D0FAD8500EE2
:10A420000001CE6FCF6B66EC55F00001CD07CCA1DB
:10A4300002D0F2D801D0F3D8E9D80001D890CC33BB
:10A44000500ECE6FCF6B66EC55F0E4D7E2D8E4D86F
:10A45000880E006E130E016E000E026E036E80B643
:10A46000FED70006000E015A025A035A035000108C
:10A4700001100210D8A402D0118C000C640E00014F
:10A48000CE6FCF6B66EC55F0010CC9000001CB6BB1
:10A490000001CB51C925006E000ECA21016E00C01B
:10A4A000F6FF01C0F7FF0F0EF76403D00800F55068
:10A4B00005D0F6CFE9FFF7CFEAFFEF500009D8B497
:10A4C00012000001CB51C925006E000ECA21016E99
:10A4D00000C0F6FF01C0F7FF0F0EF76403D00800BD
:10A4E000F55005D0F6CFE9FFF7CFEAFFEF504FDF89
:10A4F0000001CB2BCDD7D96E0A0E016ED950D1EC0D
:10A5000007F0300F0001BB6FD950BA6FBB513FDF6E
:10A510000A0E016E0001BA51D1EC07F00050300F65
:10A52000BB6FBB5134D780A4FED776D83C0E000158
:10A53000CE6FCF6B66EC55F06CD83C0E0001CE6F41
:10A54000CF6B66EC55F0010C6AD83C0E0001CE6F63
:10A55000CF6B66EC55F05AD83C0E0001CE6FCF6B36
:10A5600066EC55F080A4010CFDD7BA00C80E0001BE
:10A57000CE6FCF6B66EC55F081A002D04DD8000CA9
:10A580004ED80001BC5192DEBAC0E9FFBBC0EAFF61
:10A59000EF6EBAC0E1FFBBC0E2FFE7500F0BD96E10
:10A5A00011AC81B0000CE750006E27CFE8FF200906
:10A5B0000018D8B4200CE7503F0AD8B43F0CE7503D
:10A5C000006E27CFE8FF40090018D8B4400CE750D0
:10A5D0005F0AD8B45F0CE750F00BF00AD8B4F00C67
:10A5E000E750F00BE00AD8B4E00CE750F00B600A3B
:10A5F000D8A4000CD9500F0AD8B46F0C600C81801D
:10A60000938012009350936E819012008084928404
:10A610001200929480941200808692861200929684
:10A6200080961200819C819E818A819881940A0E75
:10A6300081EC55F08184819A210E51D835CFE8FF05
:10A640004ED8060E4CD8130E4AD8200E48D80C0E01
:10A6500046D0E8D70001D76B000E37D80001F80EBE
:10A66000C06F010EC16F0001C051006EC151016E7B
:10A67000C007000EC15B01500010D8B41200000EDC
:10A6800054D8F1D70001D76B000E1FD80001AB6B77
:10A69000AC6B660EF66E170EF76E0800F55045D8D7
:10A6A0000001AC05F80ED8B4AB19D8B41200AB4B0E
:10A6B000AC2BAB51660FF66EAC51F76E170EF7224E
:10A6C0000800F55032D8ECD7D7000001D86FD85128
:10A6D000060DF350800F03D80001D751400FE96EEB
:10A6E0008198E950E16E080ED96ED950D8B41200A5
:10A6F000819C010EE8CF20FA0A0100F000F0202F23
:10A700007DEF53F0D906E1AE02D0818E01D0819E5B
:10A71000818C010EE8CF20FA0A0100F000F0202F12
:10A720008DEF53F0D890E136E0D7E96E8188D9D724
:10A730001184120011921194120011821200006E05
:10A7400011A208D0400E006405D05B0E006002D05C
:10A75000400E00260050050DF350660FF66EF450C3
:10A76000F76E120E11B445D0F7220800F550DDDF68
:10A770000050050DF350660FF66EF450F76E120E92
:10A78000F722F62A000EF7220800F550CEDF00501F
:10A79000050DF350660FF66EF450F76E120EF722A9
:10A7A000020EF626000EF7220800F550BEDF00501C
:10A7B000050DF350660FF66EF450F76E120EF72289
:10A7C000030EF626000EF7220800F550AEDF00500B
:10A7D000050DF350660FF66EF450F76E120EF72269
:10A7E000040EF626000EF7220800F5509EDF000E3C
:10A7F0009CD7F7220800F550FE0897DF0050050DA2
:10A80000F350660FF66EF450F76E120EF722F62A2A
:10A81000000EF7220800F550FE0887DF0050050DF6
:10A82000F350660FF66EF450F76E120EF722020E1A
:10A83000F626000EF7220800F550FE0876DF0050DD
:10A84000050DF350660FF66EF450F76E120EF722F8
:10A85000030EF626000EF7220800F550FE0865DF0D
:10A860000050050DF350660FF66EF450F76E120EA1
:10A87000F722040EF626000EF7220800F550FE0817
:10A8800054DFFE0E52D7D700D96ED7C002F0036A4C
:10A89000D950520DF3CF00F0F4CF01F02AEC57F06D
:10A8A00004C0F6FF05C0F7FF7E0E3FDF520EF36EC9
:10A8B000F46AF350006EF450016EF306000EF45A81
:10A8C00001500010D8B411D0F750F45C02E1F650FA
:10A8D000F35CD8A004D00001D751D8A403D0420E15
:10A8E00024DFE7D77E0E21DFE4D77E0E1ED7A5003A
:10A8F000A5C0A5F0A6C0A6F00001A5515E0FF66E9A
:10A90000A651F76E190EF7220800F550BB6E080E1F
:10A91000D96E0001A851A65D02E1A751A55DD8B08E
:10A9200012000001A54BA62BA5515E0FF66EA65195
:10A93000F76E190EF7220800F550BB6E550ECE6F5C
:10A94000CF6B66EC55F0E5D7A5000001A507D8A0B0
:10A95000A607A56BA66B320EA76F540E46D000015A
:10A96000A56BA66BD00EA76F070EA86FC1DF000105
:10A97000900EC06F010EC16FA5EC55F00001A56BE4
:10A98000A66BD00EA76F070EA86FB2DF640E81EC26
:10A9900055F00001A56BA66BD00EA76F070EA86F30
:10A9A000A7DFC80E81EC55F00001A56BA66BD00E99
:10A9B000A76F070EA86F9CDF320E81EC55F00001E7
:10A9C000A56BA66BD00EA76F070E0FD00001A56B6D
:10A9D000A66B930EA76F120E08D000011C0EA56F78
:10A9E0000C0EA66F040EA76F100EA86F81D7BA00C9
:10A9F0000001BE51006EBF51016EBE07000EBF5B6D
:10AA000001500010D8B45ED0BAC0F6FFBBC0F7FF4B
:10AA10000F0EF76403D00800F55005D0F6CFE9FF1C
:10AA2000F7CFEAFFEF500009D8B422D0BCC0F6FF40
:10AA3000BDC0F7FF0F0EF76403D00800F55005D036
:10AA4000F6CFE9FFF7CFEAFFEF50006EBAC0F6FF8E
:10AA5000BBC0F7FF0F0EF76403D00800F55005D018
:10AA6000F6CFE9FFF7CFEAFFEF500018D8B424D0B3
:10AA7000BAC0F6FFBBC0F7FF0F0EF76403D00800A3
:10AA8000F55005D0F6CFE9FFF7CFEAFFEF50006EA3
:10AA9000016ABCC0F6FFBDC0F7FF0F0EF76403D01C
:10AAA0000800F55005D0F6CFE9FFF7CFEAFFEF50E9
:10AAB000005E000E015A12000001BA4BBB2BBC4BCA
:10AAC000BD2B96D7006A016A1200CE000001CF515B
:10AAD000D96E0BD0D906FD0EE8CF20FA0A0100F09E
:10AAE00000F0202F6FEF55F00400010ED960F2D76F
:10AAF000CEC020FA0A0100F000F0202F7BEF55F0C5
:10AB00001200E16E040ED96EFA0EE8CF20FA0A01A7
:10AB100000F000F0202F88EF55F00400D92EF4D774
:10AB2000E12EF0D71200E16E040ED96EFA0EE8CFD6
:10AB300020FA0A0100F000F0202F9AEF55F0D92EEC
:10AB4000F5D7E12EF1D71200C000040ED96EFA0E2F
:10AB5000E8CF20FA0A0100F000F0202FABEF55F00B
:10AB60000400D92EF4D7C00EE96E000EEA6EEE0690
:10AB7000000EED5AEE50ED10D8B41200E6D7F36E89
:10AB8000040EE96EFA0EBDDF0400E92EFBD7F32EAA
:10AB9000F7D712000F0E806E816A440E826E3D0E52
:10ABA000926E010E936E930E946E010EC26E0E0E97
:10ABB000C16E860EC06EC79EC79CC688C696C694D8
:10ABC000C682C690C68A0A0EAF6E240EAC6E900E78
:10ABD000AB6EF28AD76AD66AD59CD59AD596D584BB
:10ABE000D582D5809D909F80CF6ACE6ACD8CCD9A3C
:10ABF000CD98CD96CD84CD92CD90CB68BB6A040E16
:10AC0000CA6E0C0EBA6EF19CF288D08EF28CF28E67
:10AC100012000001EC6F0AD0ACA2FED70001EC518B
:10AC2000AD6E12000001EC519FEF53F0000E11B019
:10AC3000010E026E036A05D00250EEE0010AF2E056
:10AC400012000350F9E01200C96EC7A0FED7C95028
:10AC50001200E96AEA6A0C6A086A096A0A6A0B6AF7
:10AC6000045005100610071006E1046A056A066A1A
:10AC7000076A3FEF57F0C00E0C1606D0D890043686
:10AC80000536063607360C2A07AEF8D70C2AD890B8
:10AC9000083609360A360B360750035C08E10650C1
:10ACA000025C05E10550015C02E10450005C09E32F
:10ACB00008800450005E0550015A0650025A0750A1
:10ACC000035AD89007320632053204320C060C5073
:10ACD0003F0BDDE10CBC8CEC57F00050046E0150D2
:10ACE000056E0250066E0350076E0850006E095044
:10ACF000016E0A50026E0B50036E0CAE43EF57F01C
:10AD00008CEC57F043EF57F0E96AEA6A0050086E9E
:10AD10000150096E02500A6E03500B6E026A036AFC
:10AD200008500402F3CF00F0F4CF01F00502F35015
:10AD30000126F450022209500402F3500126F45077
:10AD40000222D8B0032A08500602F3500226F4501B
:10AD5000032209500502F3500226F45003220A5040
:10AD60000402F3500226F450032208500702F35065
:10AD7000032609500602F35003260A500502F35039
:10AD800003260B500402F350032643EF57F0066AE4
:10AD9000046A056A0250031003E1006A016A000CAC
:10ADA0001F0E0612D890062A02360336FCE3033241
:10ADB00002320250005C0350015804E3016E02505D
:10ADC000005ED88004360536062E06BAF0D706AEE9
:10ADD00005D0041E042AD8B40506051E0450026ED0
:10ADE0000550036E06AC000C001E002AD8B4010604
:10ADF000011E000C08EC00F0AA6A010EA96E3F0EBD
:10AE0000A616A680A8CF35FF800E0F01356101D0B0
:10AE100005D035CF00F00028D8A41200BB0EE8CF33
:10AE200035FF120008EC00F0AA6A010EA96E35CFBA
:10AE3000A8FF3F0EA616D890F2BED880F29EA68438
:10AE4000550EA76EAA0EA76EA682A198A694D8B09A
:10AE5000F28E1200066A01AE06D0001E004A0106FC
:10AE6000011E068C068E0350800B061A03AEC8EF37
:10AE700056F0021E024A0306031EC8EF56F0036A8C
:10AE8000026A016A006AE950EA1008E003C0EDFFB7
:10AE900002C0EDFF01C0EDFF00C0EFFF000C02504B
:10AEA0000002F3CF04F0F4CF05F00102F3500526C1
:10AEB00003500002F35005261200C5000001C5C072
:10AEC00000F0C6C001F0C6AF1200001E011E002A2D
:10AED000D8B4012A1200046E042A0406D8B4000C67
:10AEE000D8900036013602360336F7D7046E042AAE
:10AEF0000406D8B4000CD89003320232013200327A
:10AF0000F7D7DFC0E1F0E0C0E2F0000EE8CFDFF0FD
:10AF1000E8CFE0F02BEF4FF0001E011E021E031ED3
:10AF2000000E002A0122022203221200EE6AEA50D9
:10AF3000E262FCD7E950E162F9D71200FFFFFFFFA0
:10AF4000FFFFFFFFFFFFFFFFFFFFFFFFFFFFFFFF11
:10AF5000FFFFFFFFFFFFFFFFFFFFFFFFFFFFFFFF01
:10AF6000FFFFFFFFFFFFFFFFFFFFFFFFFFFFFFFFF1
:10AF7000FFFFFFFFFFFFFFFFFFFFFFFFFFFFFFFFE1
:10FF3000FFFFFFFFFFFFFFFF10EF00F0FFFFFFFFDE
:10FF400082B2FAD7240EAC6E0A0EAF6E900EAB6E74
:10FF500046D8C10853E14F0EAD6E4B0EAD6E006A30
:10FF60003ED8F86E076E3BD8F76EA96E38D8F66E9D
:10FF7000A86E35D8016E012A00EE09F0F56E2FD873
:10FF8000EC6E012EFBD700661FD007AC03D0040E29
:10FF90001ED818D007AE04D00C00C40E18D812D04A
:10FFA000940E15D80A00080E056E00EE0AF0080E31
:10FFB000066EEE50F56E0F00062EFBD7840E07D8A6
:10FFC000052EF5D7A694C9D74E0EAD6EC8D7A66E2E
:10FFD000550EA76EAA0EA76EA68200001200370E5D
:10FFE000026E036A046A9EAA03D0AE500026120075
:10FFF000042EF9D7032EF6D7022EF3D7AB9E9CD74B
:0200000400F00A
:10000000FFFFFFFFFFFFFFFFFFFFFFFFFFFFFFFF00
:10001000FFFFFFFFFFFFFFFFFFFFFFFFFFFFFFFFF0
:10002000FFFFFFFFFFFFFFFFFFFFFFFFFFFFFFFFE0
:10003000FFFFFFFFFFFFFFFFFFFFFFFFFFFFFFFFD0
:020000040030CA
:0E0000000002161E008081000FC00FE00F40AE
:020000040020DA
:08000000FFFFFFFFFFFFFFFF00
:00000001FF
